:020000040800F2
:1000000000000220D1410008754000087740000838
:10001000794000087B4000087D4000080000000097
:100020000000000000000000000000008127000820
:100030007F400008000000002128000881400008DF
:100040002142000821420008214200082142000804
:1000500021420008214200082142000821420008F4
:1000600021420008214200082142000821420008E4
:1000700021420008214200082142000821420008D4
:1000800021420008214200082142000821420008C4
:1000900021420008214200082142000821420008B4
:1000A00021420008214200082142000821420008A4
:1000B0002142000821420008214200082142000894
:1000C0002142000821420008214200082142000884
:1000D0002142000821420008214200082142000874
:1000E0002142000821420008214200082142000864
:1000F0002142000821420008214200082142000854
:100100002142000821420008214200082142000843
:100110002142000821420008214200082142000833
:100120002142000821420008214200082142000823
:100130002142000821420008214200082142000813
:100140002142000821420008214200082142000803
:1001500021420008214200082142000821420008F3
:1001600021420008214200082142000821420008E3
:10017000214200082142000821420008000000003E
:080180002142000821420008A1
:1001900010B5054C237833B9044B13B10448AFF3C1
:1001A00000800123237010BD7C00002000000000AF
:1001B0009056000808B5034B1BB103490348AFF341
:1001C000008008BD0000000080000020905600085C
:1001D000034613F8012B002AFBD1181A0138704787
:1001E00001F0FF01102A2BDB10F0070F08D010F8E8
:1001F000013B013A8B422DD010F0070F42B3F6D1EC
:10020000F0B441EA012141EA014122F007047FF004
:1002100000070023F0E80256083C85EA010586EA5B
:10022000010685FA47F5A3FA87F586FA47F6A5FA97
:1002300087F68EB9EED1F0BC01F0FF0102F00702A3
:1002400032B110F8013B013A83EA010313B1F8D14E
:100250000020704701387047002D06BF354603382F
:10026000073815F0010F07D1013015F4807F02BF68
:10027000013015F4C03F0130F0BC0138704700BFB9
:1002800053B94AB9002908BF00281CBF4FF0FF31FD
:100290004FF0FF3000F088B9ADF1080C6DE904CEE5
:1002A00000F006F8DDF804E0DDE9022304B0704751
:1002B0002DE9F047089D8E4604468846002B4AD11A
:1002C0008A42174662D9B2FA82F64EB1C6F12003CD
:1002D00001FA06F820FA03F3B74043EA0808B440ED
:1002E0004FEA174E1FFA87FCB8FBFEF1230C0EFBFA
:1002F000118843EA084301FB0CF29A4209D9FB1822
:1003000001F1FF3080F0EA809A4240F2E780023942
:100310003B449A1AA3B2B2FBFEF00EFB102243EA52
:10032000024300FB0CFC9C4509D9FB1800F1FF328D
:1003300080F0D6809C4540F2D3803B44023840EAAE
:100340000140A3EB0C0300211DB1F3400022C5E9DD
:100350000032BDE8F0878B4205D90DB1C5E9000137
:1003600000210846F5E7B3FA83F1002946D1734529
:1003700002D3824200F20581841A6EEB030201204F
:100380009046002DE5D0C5E90048E2E7002A00F0DC
:100390009080B2FA82F6002E40F0A4808A1A030CF4
:1003A0004FEA174E80B2BCB20121B2FBFEFC0EFB3D
:1003B0001C2243EA024304FB0CF29A4207D9FB18C1
:1003C0000CF1FF3802D29A4200F2E080C4469B1A38
:1003D000B3FBFEF20EFB123340EA034302FB04F4CC
:1003E0009C4207D9FB1802F1FF3002D29C4200F276
:1003F000CA8002461B1B42EA0C40A5E7C1F1200659
:100400008B4022FA06F71F430EFA01F420FA06F396
:100410002EFA06FE4FEA1749234300FA01F81FFAA5
:1004200087FCBEFBF9F01C0C09FB10EE44EA0E44FD
:1004300000FB0CFEA64502FA01F209D93C1900F1B5
:10044000FF3A80F09C80A64540F2998002383C44F7
:10045000A4EB0E041FFA83FEB4FBF9F309FB13446B
:100460004EEA044403FB0CFCA44508D93C1903F1F3
:10047000FF3E80F08280A4457FD9023B3C4443EAA2
:100480000040A4EB0C04A0FB02EC64457346E1467B
:1004900062D35FD05DB1B8EB030264EB090404FAE8
:1004A00006F622FA01F31E43CC40C5E900640021A0
:1004B0004FE7B1FBF2FC010C41EA0E4180B240EA89
:1004C00001423B4638463C46B846BE462026B1FB74
:1004D000F7F1A2EB080241EA0C4166E7014618E792
:1004E00010462CE7C6F120022EFA02F3B740B140C5
:1004F00020FA02F24FEA174E0A43B3FBFEF8BCB2F1
:100500000EFB1833110C41EA034108FB04F9B0401B
:1005100089454FEA104380B23ED9791808F1FF3C73
:1005200001D289451FD8A1EB0901B1FBFEF909FBF6
:1005300004F80EFB191192B242EA0142424529D257
:10054000BA1809F1FF31C4D24245C2D2A9F1020161
:100550003A44BEE7F0459DD2BEEB02036CEB070CBC
:100560000138E14696E7A7EB09094944A8F1020CD6
:10057000B1FBFEF909FB04F8DBE773467FE7504661
:1005800066E70846FDE63B44023A33E7ACF1020C6D
:100590003B441CE749469CE7A1EB0901C446B1FB7B
:1005A000FEF909FB04F8C4E7704700BF10B5044624
:1005B0000E4B1A784FF47A73B3FBF2F30C4A1068BF
:1005C000B0FBF3F000F0ACF868B90F2C01D90120B2
:1005D0000AE0002221464FF0FF3000F091F8034B73
:1005E0005C60002000E0012010BD00BF0000002082
:1005F0002800002008B50B4B1A6842F400721A60FC
:100600001A6842F480621A601A6842F480721A60B2
:10061000032000F063F80F20FFF7C8FF03F008FD88
:10062000002008BD003C0240034A1168034B1B78C0
:100630000B441360704700BF9800002000000020AA
:10064000014B1868704700BF9800002038B5044679
:10065000FFF7F6FF0546B4F1FF3F02D0044B1B78CD
:100660001C44FFF7EDFF401BA042FAD338BD00BF8A
:1006700000000020002808DB0901C9B200F1604039
:1006800000F5614080F80013704700F00F00090189
:10069000C9B2014B1954704714ED00E000B500F0E9
:1006A0000700C0F1070CBCF1040F28BF4FF0040C89
:1006B000031D062B0FD9C31E4FF0FF3E0EFA0CF0A0
:1006C00021EA000199400EFA03FE22EA0E0241EAF5
:1006D00002005DF804FB0023EEE70000074AD36840
:1006E00023F4E0631B041B0C000200F4E0600343EE
:1006F00043F0BF6343F40033D360704700ED00E084
:1007000010B50446054BD868C0F30220FFF7C6FFBA
:1007100001462046FFF7AEFF10BD00BF00ED00E030
:100720000138B0F1807F0BD24FF0E0235861054AC9
:10073000F02182F823100020986107221A61704787
:100740000120704700ED00E000230F2B00F2E9804C
:1007500070B582B065E085684FEA430E032404FA61
:100760000EF425EA0405CC6804FA0EF42C438460E8
:10077000446824EA02044A68C2F300129A40224301
:1007800042605CE0DC08083450F8242003F00705E0
:10079000AD004FF00F0E0EFA05FE22EA0E0E0A69AA
:1007A000AA4042EA0E0240F824205CE0072200E062
:1007B000002202FA0EF22A4302345A4D45F8242050
:1007C000594A94686FEA0C0224EA0C054E6816F444
:1007D000801F01D04CEA0405534CA560E46802EA8E
:1007E00004054E6816F4001F01D04CEA04054E4C77
:1007F000E560646802EA04054E6816F4003F01D023
:100800004CEA0405484C6560246822404D6815F4A4
:10081000803F01D04CEA0402434C226001330F2B8D
:100820007DD801229A400C6804EA020C32EA0404E2
:10083000F4D14C6804F00304013C012C8BD94A68C4
:1008400002F00302032A09D0C4685D000322AA4013
:1008500024EA02048A68AA402243C2604A6802F07D
:100860000302022A8ED004684FEA430E032202FAE2
:100870000EF224EA02044A6802F0030202FA0EF2BF
:10088000224302604A6812F4403FC7D0002201921E
:10089000264A546C44F480445464526C02F48042FE
:1008A0000192019A9C08A51C1E4A52F8255003F09B
:1008B000030E4FEA8E0E0F2202FA0EF225EA02050F
:1008C0001B4A90423FF474AF02F5806290421AD006
:1008D00002F58062904218D002F58062904216D0F4
:1008E00002F58062904214D002F58062904212D0EC
:1008F00002F58062904210D002F5806290423FF48F
:1009000055AF082255E7012253E7022251E703229F
:100910004FE704224DE705224BE7062249E702B0E4
:1009200070BD704700380140003C01400038024073
:100930000000024003685A6912F4806F01D1002060
:1009400070476FF480625A6100230363202280F8AD
:100950003D2080F83E30026C42F00402026480F8D0
:100960003C30012070472DE9F04106460C46174601
:1009700098463BE0FFF764FE069BC01A404502D84C
:10098000B8F1000F32D1012D18D033689B6924EAE9
:1009900003039BB2B3FA83F35B099F4226D1002382
:1009A0003363202286F83D2086F83E30326C42F0D8
:1009B0002002326486F83C30012027E033685B690E
:1009C00024EA03039BB2B3FA83F35B09E5E73368D8
:1009D0005B6924EA030C1FFA8CFCBCFA8CFC4FEA1E
:1009E0005C1C674511D1B8F1FF3FC3D1C4F3074583
:1009F000012DECD033689B6924EA030C1FFA8CFCB0
:100A0000BCFA8CFC4FEA5C1CEBE70020BDE8F081EF
:100A10002DE9F84305460E469046994653E01A687C
:100A200042F400721A602B686FF480625A610023EE
:100A30002B63202285F83D2085F83E302A6C42F059
:100A400004022A6485F83C3001204AE0FFF7F8FDF3
:100A5000A0EB0900404502D8B8F1000F33D1012FB7
:100A600017D02B689B6926EA03039BB2003B18BF93
:100A7000012343B300232B63202285F83D2085F812
:100A80003E302A6C42F020022A6485F83C30012076
:100A900027E02B685B6926EA03039BB2003B18BF83
:100AA0000123E6E72B689C6926EA0404A4B2003C13
:100AB00018BF0124A4B12B685A6912F4806FAED11B
:100AC000B8F1FF3FC2D1C6F30747012FEAD12B6827
:100AD0005C6926EA0404A4B2003C18BF0124E9E7DB
:100AE0000020BDE8F88370B504460D46164623681D
:100AF0005B6913F0800F21D12046FFF71BFFF8B987
:100B0000B5F1FF3FF3D0FFF79BFD801BA84201D852
:100B1000002DECD123685B6913F0800FE7D100232F
:100B20002363202284F83D2084F83E30226C42F07A
:100B30002002226484F83C30012000E0002070BDD7
:100B40000120FCE72DE9F04385B004460D469146AF
:100B50001F46DDF830800D9E0368196841F48071EE
:100B600019600096434600224FF00111FFF7FBFE8B
:100B700060B9236805F0FE051D61334642462649EB
:100B80002046FFF745FF68B1012008E023681B6895
:100B900013F4807F02D04FF400732364032005B068
:100BA000BDE8F0830023039323685A6903929B698D
:100BB0000393039B324641462046FFF794FF30B92A
:100BC000012F0FD123685FFA89F61E61E7E7236CD6
:100BD000042B01D00120E2E72268136843F400737C
:100BE0001360F7E723684FEA19221A61324641463B
:100BF0002046FFF778FF20B923685FFA89F61E6167
:100C0000CDE7236C042B01D00120C8E722681368CC
:100C100043F400731360F7E7020001002DE9F04789
:100C200084B004460D46164699460C9FDDF8348084
:100C30000268136843F4806313600368196841F421
:100C400080711960CDF800803B4600224FF0011101
:100C5000FFF789FE70B95FFA85FA236805F0FE0593
:100C60001D6143463A4641492046FFF7D1FE68B12F
:100C7000012008E023681B6813F4807F02D04FF442
:100C800000732364032004B0BDE8F08700230393BE
:100C900023685A6903929B690393039B4246394632
:100CA0002046FFF720FF80B9B9F1010F18D1236862
:100CB000F6B21E61424639462046FFF714FF68B37C
:100CC000236C042B24D00120DDE7236C042B01D0FE
:100CD0000120D8E72268136843F400731360F7E734
:100CE0002368320A1A61424639462046FFF7FBFE66
:100CF00018B92368F6B21E61DCE7236C042B01D01F
:100D00000120C0E72268136843F400731360F7E71B
:100D10002268136843F400731360D4E722681368F1
:100D200043F480731360CDF800803B4600224FF0FF
:100D300001112046FFF717FE68B922684AF0010347
:100D4000136143463A4609492046FFF761FE0028F1
:100D500099D0012097E723681B6813F4807F02D0A5
:100D60004FF40073236403208DE700BF02000100ED
:100D700070B504460D46164623685B6913F0040FF0
:100D800021D12046FFF7D6FDF8B9B5F1FF3FF3D0EA
:100D9000FFF756FC801BA84201D8002DECD1236838
:100DA0005B6913F0040FE7D100232363202284F84A
:100DB0003D2084F83E30226C42F02002226484F808
:100DC0003C30012000E0002070BD0120FCE770B540
:100DD00004460D46164614E06FF010025A610023D7
:100DE0002363202284F83D2084F83E30226C226464
:100DF00084F83C30012025E023685B6913F0400F44
:100E000010D02368586910F0400F1AD1586910F0BB
:100E1000100FE1D1FFF714FC801BA842ECD8002D85
:100E2000EFD1E9E700232363202284F83D2084F8F2
:100E30003E30226C42F02002226484F83C300120D3
:100E400000E0002070BD0000002800F0CC8070B5EC
:100E5000044690F83D30002B77D0242384F83D30B1
:100E60002268136823F0010313602268136843F4B7
:100E7000004313602268136823F40043136000F0FA
:100E8000F5FD62685A4B9A4264D85A4B98428CBF1F
:100E900000230123002B40F0A8805749A1FB00311B
:100EA0008B0C25686A6822F03F0242EA91426A6030
:100EB00021680A6A22F03F0266684D4DAE424FD863
:100EC000013313430B622168CA6922F44F4222F0B6
:100ED000FF026568464B9D424CD8431E6D00B3FB34
:100EE000F5F3013340F6FC70034278D0C3F30B03F3
:100EF0001A43CA6121680B6823F0C003E269206AC3
:100F0000024313430B6021688B6823F4034323F0EF
:100F1000FF032269E068024313438B602168CB68BA
:100F200023F0FF036269A06902431343CB60226888
:100F3000136843F00103136000202064202384F829
:100F40003D30206384F83E0070BD80F83C3002F0F4
:100F5000ADFD82E7294B98428CBF0023012399E71E
:100F60004FF4967505FB03F3254DA5FB03539B0931
:100F70000133A6E7A668BEB9431E05EB450CB3FBDB
:100F8000FCF30133C3F30B03B3FA83F35B0943BBF5
:100F9000C6B9431E05EB4505B3FBF5F30133C3F3B7
:100FA0000B0343F40043A3E7431E05EB850C0CEB56
:100FB0008C0CB3FBFCF30133C3F30B03B3FA83F3E1
:100FC0005B09E4E7431E05EB850505EB8505B3FBEF
:100FD000F5F30133C3F30B0343F4404388E70423E1
:100FE00086E7012384E7012070470120ACE700BFBA
:100FF000A08601007F841E0083DE1B43FF083D00A6
:10100000D34D62102DE9F04383B004460F4690465D
:1010100099460C9EFFF714FB054694F83D00C0B2BC
:10102000202803D0022003B0BDE8F08300951923E7
:1010300001224B492046FFF796FC002840F08980AA
:1010400094F83C30012B00F08680012384F83C307A
:1010500023681A6812F0010F03D11A6842F00102E6
:101060001A602268136823F400631360212384F854
:101070003D30402384F83E30002323640A9B6362A2
:10108000BDF82C306385638D2385364BE362019573
:1010900000964B46424639462046FFF753FD00284E
:1010A0005BD1238D002B35D02A4631462046FFF7F1
:1010B0001AFD20BB626A236812781A61626A531CA7
:1010C0006362218D013989B22185638D9BB2013B19
:1010D0009BB263852368586910F0040FE1D00029A2
:1010E000DFD052781A61636A01336362238D013B5A
:1010F0002385638D9BB2013B9BB26385D1E7236C53
:10110000042B01D001208EE72268136843F400739A
:101110001360F7E72A4631462046FFF729FE50B113
:10112000236C042B01D001207DE72268136843F46F
:1011300000731360F7E72268136843F400731360C9
:10114000202384F83D30002384F83E3084F83C307E
:1011500069E7022067E7022065E7012063E700BF37
:10116000020010000000FFFF2DE9F04387B00446A5
:101170000F4690469946109EFFF762FA054694F88E
:101180003D00C0B2202804D00227384607B0BDE891
:10119000F08300951923012288492046FFF7E3FBDD
:1011A000002840F04D8194F83C30012B00F04A813A
:1011B000012384F83C3023681A6812F0010F03D130
:1011C0001A6842F001021A602268136823F400636F
:1011D0001360222384F83D30402384F83E300023FE
:1011E00023640E9B6362BDF83C306385638D238569
:1011F000734BE362019500964B46424639462046C2
:10120000FFF70CFD0746002840F01E81238D5BB9D7
:10121000029323685A6902929A690292029A1A68A2
:1012200042F400721A6075E0012B0AD0022B1AD02A
:101230000023059323685A6905929B690593059BD2
:1012400068E02268136823F480631360002303932B
:1012500023685A6903929A690392039A1A6842F4BE
:1012600000721A6056E02268136823F480631360EA
:101270002268136843F40063136000230493236817
:101280005A6904929B690493049B43E02A463146C1
:101290002046FFF79CFD002840F0D88023681A699B
:1012A000636A1A70636A01336362238D013B23858D
:1012B000638D9BB2013B9BB263852BE00095334667
:1012C000002240492046FFF74EFB002840F0C08036
:1012D0002268136843F40073136023681A69636A11
:1012E0001A70626A531C6362238D013B2385638DF0
:1012F0009BB2013B9BB2638523681B695370636A91
:1013000001336362238D013B2385638D9BB2013BD7
:101310009BB26385238D002B00F08980032B53D86B
:10132000012BB3D0022BC9D00095334600222549AA
:101330002046FFF718FB002840F08C8022681368D5
:1013400023F48063136023681A69636A1A70636AFE
:1013500001336362238D013B2385638D9BB2013B87
:101360009BB2638500953346002216492046FFF75D
:10137000FAFA002870D12268136843F400731360EE
:1013800023681A69636A1A70626A531C6362238D48
:10139000013B2385638D9BB2013B9BB26385236830
:1013A0001B695370636A01336362238D013B23859C
:1013B000638D9BB2013B9BB26385ABE702001000DB
:1013C0000000FFFF040001002A4631462046FFF7D7
:1013D000FEFC002842D123681A69636A1A70636AA6
:1013E00001336362228D013A92B22285638D9BB2F2
:1013F000013B9BB263852368596911F0040F89D0C2
:10140000032A0FD023681A69636A1A70636A01336A
:101410006362238D013B2385638D9BB2013B9BB2AD
:10142000638577E71A6822F480621A60EAE720236E
:1014300084F83D30002384F83E3084F83C30A4E644
:101440000227A2E60227A0E601279EE601279CE6E6
:1014500001279AE6012798E6012796E6012794E6F8
:10146000002800F0E08170B582B00446036813F0F4
:10147000010F3BD09F4B9B6803F00C03042B2CD037
:101480009C4B9B6803F00C03082B21D06368B3F5D9
:10149000803F4FD0B3F5A02F52D0964B1A6822F45C
:1014A00080321A601A6822F480221A606368002B66
:1014B00050D0FFF7C5F805468E4B1B6813F4003F6C
:1014C00014D1FFF7BDF8401B6428F5D90320B1E122
:1014D000884B5B6813F4800FD8D0864B1B6813F4DD
:1014E000003F03D06368002B00F09F81236813F056
:1014F000020F54D07F4B9B6813F00C0F3ED07D4BF6
:101500009B6803F00C03082B33D0E368002B68D0F2
:10151000794B01221A60FFF793F80546754B1B685B
:1015200013F0020F54D1FFF78BF8401B0228F5D9B6
:1015300003207FE16F4A136843F480331360B5E7FB
:101540006C4B1A6842F480221A601A6842F48032A6
:101550001A60ABE7FFF774F80546664B1B6813F497
:10156000003FC3D0FFF76CF8401B6428F5D9032077
:1015700060E1604B5B6813F4800FC6D15D4B1B6864
:1015800013F0020F03D0E368012B40F05081594A59
:10159000136823F0F803216943EAC1031360236849
:1015A00013F0080F42D063696BB3534B0122C3F8A9
:1015B000802EFFF745F805464E4B5B6F13F0020F88
:1015C00034D1FFF73DF8401B0228F5D9032031E163
:1015D000484A136823F0F803216943EAC103136002
:1015E000DDE7454B00221A60FFF72AF80546414B1C
:1015F0001B6813F0020FD2D0FFF722F8401B02281D
:10160000F5D9032016E13C4B0022C3F8802EFFF7EA
:1016100017F80546374B5B6F13F0020F06D0FFF744
:101620000FF8401B0228F5D9032003E1236813F0CB
:10163000040F77D02F4B1B6C13F0805F33D1002346
:1016400001932C4B1A6C42F080521A641B6C03F00D
:1016500080530193019B0125284B1B6813F4807F65
:1016600023D0A368012B34D0052B38D0214B1A6F1F
:1016700022F001021A671A6F22F004021A67A368A7
:10168000002B3DD0FEF7DCFF06461A4B1B6F13F014
:10169000020F46D1FEF7D4FF801B41F288339842F7
:1016A000F3D90320C6E00025D6E7144A136843F4B3
:1016B00080731360FEF7C4FF0646104B1B6813F4DB
:1016C000807FCED1FEF7BCFF801B0228F5D9032016
:1016D000B0E0084A136F43F001031367CFE7054BEF
:1016E0001A6F42F004021A671A6F42F001021A6779
:1016F000C5E700BF003802400000474200700040CC
:10170000FEF79EFF0646524B1B6F13F0020F08D0E8
:10171000FEF796FF801B41F288339842F3D90320ED
:1017200088E0EDB9A369002B00F08380484A9268F5
:1017300002F00C02082A51D0022B17D0454B002290
:101740001A66FEF77DFF0446414B1B6813F0007FCD
:1017500042D0FEF775FF001B0228F5D9032069E08F
:101760003B4A136C23F080531364DBE7394B0022B0
:101770001A66FEF765FF0546354B1B6813F0007FC0
:1017800006D0FEF75DFF401B0228F5D9032051E08B
:10179000E369226A1343626A43EA8213A26A520827
:1017A000013A43EA0243E26A43EA0263284A536089
:1017B000284B01221A66FEF743FF0446244B1B68A0
:1017C00013F0007F06D1FEF73BFF001B0228F5D97E
:1017D00003202FE000202DE000202BE0012B2BD058
:1017E0001B4B5B6803F48001E269914226D103F050
:1017F0003F02216A8A4223D1616A47F6C0721A40C9
:10180000B2EB811F1ED103F44031A26A5208013AA3
:10181000B1EB024F18D103F07063E26AB3EB026FD1
:1018200014D1002006E001207047012002E00120D1
:1018300000E0002002B070BD0120FBE70120F9E7C5
:101840000120F7E70120F5E70120F3E70120F1E7A8
:10185000003802400000474208B5264B9B6803F061
:101860000C03042B41D0082B41D1224B5A6802F0C3
:101870003F025B6813F4800F12D01E4B5968C1F30E
:1018800088111D480023A1FB0001FEF7F9FC194B4C
:101890005B68C3F3014301335B00B0FBF3F008BDA9
:1018A000144B5868C0F388104FEA401CBCEB000C86
:1018B0006EEB0E0E4FEA8E1343EA9C634FEA8C11D7
:1018C000B1EB0C0163EB0E03DB0043EA5173C9007B
:1018D00011EB000C43F10003990200234FEA8C2026
:1018E00041EA9C51FEF7CCFCD1E70348D7E7034817
:1018F000D5E700BF0038024040787D010024F400A5
:10190000002800F09B8070B50D4604464F4B1B68C5
:1019100003F007038B4208D2CBB24C4A1370136812
:1019200003F007038B4240F08B80236813F0020F13
:1019300017D013F0040F04D0454A936843F4E053E2
:101940009360236813F0080F04D0414A936843F46E
:10195000604393603E4A936823F0F003A1680B4311
:101960009360236813F0010F32D06368012B21D0FC
:101970009A1E012A25D9364A126812F0020F61D048
:1019800033498A6822F0030213438B60FEF758FE46
:1019900006462F4B9B6803F00C036268B3EB820F83
:1019A00016D0FEF74DFE801B41F288339842F0D9E5
:1019B000032042E0264A126812F4003FE0D10120E1
:1019C0003BE0234A126812F0007FD9D1012034E0B5
:1019D0001E4B1B6803F00703AB4207D9EAB21B4B4F
:1019E0001A701B6803F00703AB422DD1236813F074
:1019F000040F06D0164A936823F4E053E1680B43C2
:101A00009360236813F0080F07D0114A936823F4FA
:101A10006043216943EAC1039360FFF71DFF0C4B4C
:101A20009B68C3F303130B4AD35CD8400A4B18607E
:101A30000A4B1868FEF7BAFD002070BD0120704700
:101A40000120FAE70120F8E70120F6E7003C024018
:101A500000380240087F0008280000200400002011
:101A6000014B1868704700BF2800002008B5FFF739
:101A7000F7FF044B9B68C3F38223034AD35CD8402F
:101A800008BD00BF00380240187F000808B5FFF706
:101A9000E7FF044B9B68C3F34233034AD35CD8404F
:101AA00008BD00BF00380240187F0008026802F13C
:101AB0000C0353E8003F23F490730C3242E80031EA
:101AC0000029F3D1026802F1140353E8003F23F028
:101AD0000103143242E800310029F3D1036B012BDA
:101AE00005D0202380F8423000230363704702684A
:101AF00002F10C0353E8003F23F010030C3242E8DC
:101B000000310029F3D1ECE710B5044602681369EF
:101B100023F44053C1680B431361836802691A437D
:101B200043691A43C3691A430168CB6823F4164317
:101B300023F00C031343CB600268536923F4407312
:101B400081690B4353610368314A934206D002F521
:101B50008062934202D0FFF789FF01E0FFF796FF12
:101B6000E369B3F5004F29D00021031849411B1840
:101B700041F10001C90041EA5371DB0018186368A4
:101B80004FEA83024FEA937341F10001FEF778FBBD
:101B9000204AA2FB00314909642303FB11031B0106
:101BA0003233A2FB03235B0903F0F00202EB0112C4
:101BB00003F00F03216813448B6010BD002302184B
:101BC00043EB0301121841F10001C90041EA5271CF
:101BD000D200101841F10001626892185B41FEF7D3
:101BE0004FFB0C4AA2FB00314909642303FB11039C
:101BF000DB003233A2FB03235B095A0002F4F872C4
:101C000002EB011203F00703216813448B60D4E751
:101C1000001001401F85EB512DE9F04383B00546CC
:101C20000E4617469946DDF828802B681C6836EA70
:101C300004040CBF01240024BC4228D1B8F1FF3FAA
:101C4000F3D0FEF7FDFCA0EB0900404523D8B8F126
:101C5000000F22D02B68DA6812F0040FE5D0802E36
:101C6000E3D0402EE1D01A6812F0080FDDD0002436
:101C700001941A6801925B680193019B2846FFF763
:101C800015FF08236B6485F84040012000E0002028
:101C900003B0BDE8F0830320FAE70320F8E760B360
:101CA00010B5044690F8413013B3242384F8413032
:101CB0002268D36823F40053D3602046FFF724FF43
:101CC0002268136923F4904313612268536923F057
:101CD0002A0353612268D36843F40053D360002081
:101CE0006064202384F8413084F84230606310BD82
:101CF00080F8403002F034FAD7E7012070472DE930
:101D0000F04182B01E4690F84130DBB2202B56D114
:101D100004460D469046002955D00AB901204FE0EF
:101D200000234364212380F84130FEF789FC0746F5
:101D3000A4F82480A4F82680A368B3F5805F02D0BD
:101D40004FF0000814E023692BB34FF000080FE0B8
:101D5000202384F84130032032E038F8023B226827
:101D6000C3F308035360E28C92B2013A92B2E28468
:101D7000E38C9BB293B100963B4600228021204623
:101D8000FFF74AFF0028E3D1002DE6D015F8012B1C
:101D900023685A60E7E7A8460025E9E700963B4636
:101DA000002240212046FFF737FF18B9202384F88E
:101DB000413005E0202384F84130032000E0022078
:101DC00002B0BDE8F0810120FAE7842801D0033099
:101DD00070470020704708B500F066FA002008BD83
:101DE0002DE9F04387B00E464469C4B18569B5B1A9
:101DF0004768D0F80080D0F81090B0F90800FFF7DD
:101E0000E4FF02950194009033464A464146384625
:101E100000F0DCF90590059807B0BDE8F083446850
:101E200005680769B0F90800FFF7CFFF05AB01931C
:101E300000903346BAB22946204600F002FA012843
:101E4000E9D00020E8E708B500B9012000F0C6FBA2
:101E5000002008BD00F1080343604FF0FF328260AC
:101E6000C360036100230360704700230361704770
:101E700043684B609A688A605160996008610368A2
:101E800001330360704730B40D68B5F1FF3F11D0E6
:101E900000F108031C465B681A68AA42FAD9636815
:101EA0004B6099608C606160086103680133036076
:101EB00030BC70470469F2E70369416882688A6050
:101EC000416851605A68824206D0002202611A6855
:101ED000013A1A601868704782685A60F5E7000096
:101EE000074B9B6A1B6823B9054B4FF0FF32DA6240
:101EF0007047034B9A6AD268D2685268DA627047B8
:101F00009C0000202DE9F04707469846089DDDF823
:101F100024900A9C266B02F18042013A06EB82066D
:101F200026F00706C1B308464FF0000CBCF10F0FB6
:101F300009D810F80C2004EB0C0383F8342012B1FC
:101F40000CF1010CF2E7002384F84330062D00D990
:101F50000625E56265644FF0000AC4F848A0201D1C
:101F6000FFF783FF04F11800FFF77FFF2461C5F13D
:101F70000705A5616462C4F84CA084F850A04246ED
:101F80003946304600F0E6FB2060B9F1000F01D081
:101F9000C9F80040BDE8F087002384F83430D5E765
:101FA00070B5002407E004EB840293001048184445
:101FB000FFF750FF0134062CF5D90E4C04F1BC0696
:101FC0003046FFF747FF04F1D0052846FFF742FFF0
:101FD00004F11400FFF73EFF04F1E400FFF73AFFBD
:101FE0002046FFF737FFA662C4F8F85070BD00BF67
:101FF000CC0000209C00002038B5054600F0D2FB44
:10200000274BD3F8FC200132C3F8FC20D3F8003171
:1020100073B1234BD3F804318BB9214BD3F8003182
:10202000DA6AEB6A9A420AD81D4BC3F8005106E0FF
:102030001B4BC3F80051D3F8FC30012B2CD0184CAB
:10204000D4F808310133C4F80831EB6A01229A4010
:10205000D4F80C110A43C4F80C2104F1300003EB4E
:102060008303291D00EB8300FFF702FF00F0BCFB98
:10207000D4F804317BB1D4F80031DA6AEB6A9A42C1
:1020800009D24FF0E0234FF08052C3F8042DBFF384
:102090004F8FBFF36F8F38BDFFF782FFCFE700BFD1
:1020A0009C00002010B5044690F8513063B1012B1C
:1020B00011D0022B0ED04FF0500383F31188BFF3E1
:1020C0006F8FBFF34F8FFEE7006B00F05BFD204684
:1020D00000F058FD10BD00F055FDFBE738B517E0E6
:1020E00000F060FB0D4CD4F8F030DD68281DFFF7E0
:1020F000E3FED4F8FC30013BC4F8FC30D4F81031D6
:10210000013BC4F8103100F06FFB2846FFF7CAFF0F
:10211000024BD3F81031002BE2D138BD9C000020D7
:1021200008B5FFF7DBFF074B1B6B012BF9D94FF00D
:10213000E0234FF08052C3F8042DBFF34F8FBFF35D
:102140006F8FEEE79C00002070B504460D461E4BD5
:10215000D3F81461D3F800010430FFF7ADFE58B98D
:10216000194BD3F80021D26A01219140D3F80C21F8
:1021700022EA0102C3F80C21B4F1FF3F0FD034442E
:10218000114BD3F800315C60A64211D90E4BD3F845
:10219000F800D3F800110431FFF775FE70BD002D73
:1021A000EDD00948D0F800110431FFF761FEF5E7E2
:1021B000054DA86AD5F800110431FFF764FEEB6AFB
:1021C000A342EBD9EC62E9E79C00002030B587B070
:1021D0000B9C7CB10C9DB5B154250495049D542DE8
:1021E0001AD04FF0500383F31188BFF36F8FBFF302
:1021F0004F8FFEE74FF0500383F31188BFF36F8FCB
:10220000BFF34F8FFEE74FF0500383F31188BFF306
:102210006F8FBFF34F8FFEE7049D0C9D2C6302244C
:1022200085F8514000240394029505AC01940A9C62
:102230000094FFF767FE0C98FFF7DEFE059807B0E5
:1022400030BD2DE9F04385B00746884614461E464A
:10225000900000F021FC08B38146542000F01CFCE3
:102260000546A8B1C0F83090002380F851300393A0
:1022700002900D9B01930C9B0093334622464146EE
:102280003846FFF73FFE2846FFF7B6FE012007E07D
:10229000484600F077FC4FF0FF3001E04FF0FF3090
:1022A00005B0BDE8F083000010B588B000240594A7
:1022B000069407AA06A905A800F0A2FC059B0293B4
:1022C000069B019300942346079A0E490E48FFF798
:1022D0007DFF0E4BC3F81C0190B14FF0500383F308
:1022E0001188BFF36F8FBFF34F8F084B4FF0FF3252
:1022F000DA620122C3F80421C3F8144100F0ECFAB9
:1023000008B010BD207F0008212100089C0000209B
:10231000034AD2F818310133C2F81831704700BFB0
:102320009C000020014BD3F8140170479C00002052
:102330002DE9F041434BD3F81831002B76D1414BB6
:10234000D3F814610136C3F81461CEB99B6A1B68D7
:1023500043B14FF0500383F31188BFF36F8FBFF386
:102360004F8FFEE7374B9A6AD3F8F8109962C3F89B
:10237000F820D3F820210132C3F82021FFF7B0FD67
:10238000304BDB6AB34246D94FF000082D4AD2F8F1
:102390000031DB6A03EB830399000A44136B012BC2
:1023A00001D94FF00108274BD3F82431002B45D039
:1023B0004FF0010842E04FF00108224B9B6A1B6876
:1023C00063B3204B9B6ADB68DC6863689E422AD358
:1023D000271D3846FFF770FDA36A1BB104F11800F2
:1023E000FFF76AFDE36A01229A40164DD5F80C11F9
:1023F0000A43C5F80C2105F1300003EB83039A0072
:1024000039461044FFF734FDE26AD5F80031DB6A43
:102410009A42D0D2D1E74FF00008CEE7094B4FF0F7
:10242000FF32DA62B2E7074AD362AFE7054AD2F871
:1024300028310133C2F828314FF000084046BDE88A
:10244000F08100BF9C0000203A4BD3F8183143B90B
:102450004FF0500383F31188BFF36F8FBFF34F8F9B
:10246000FEE770B500F09EF9324BD3F81821013A1F
:10247000C3F81821D3F81831002B56D12D4BD3F8BF
:10248000FC300BB9002451E000252A4B5B692BB3CB
:10249000284C236ADD6805F11800FFF70DFD2E1D9D
:1024A0003046FFF709FDEB6A01229A40D4F80C117F
:1024B0000A43C4F80C2104F1300003EB83033146D6
:1024C00000EB8300FFF7D4FCEA6AD4F80031DB6A42
:1024D0009A42DAD30122C4F82421D6E70DB1FFF7DE
:1024E000FFFC144BD3F828418CB9124BD3F824418C
:1024F000E4B14FF0E0234FF08052C3F8042DBFF356
:102500004F8FBFF36F8F012410E0013C08D0FFF71D
:102510000FFF0028F9D0074B0122C3F82421F4E76C
:10252000044B0022C3F82821DFE7002400F05CF907
:10253000204670BD9C00002038B558B10C460546B9
:1025400089B94FF0500383F31188BFF36F8FBFF346
:102550004F8FFEE74FF0500383F31188BFF36F8F67
:10256000BFF34F8FFEE71C4BD3F8183143B14FF048
:10257000500383F31188BFF36F8FBFF34F8FFEE7D4
:10258000FFF7C6FE144BD3F814012B681C4483429A
:1025900009D9A34201D82C600EE0A04201D32C60DF
:1025A0000AE02C6004E0A34201D8A04212D22C60C1
:1025B0000021201AFFF7C8FDFFF746FF48B94FF08A
:1025C000E0234FF08052C3F8042DBFF34F8FBFF3C9
:1025D0006F8F38BD2C60EFE79C00002010B5B0B1C4
:1025E0000446104BD3F8183143B14FF0500383F336
:1025F0001188BFF36F8FBFF34F8FFEE7FFF788FEA1
:1026000000212046FFF7A0FDFFF71EFF48B94FF05D
:10261000E0234FF08052C3F8042DBFF34F8FBFF378
:102620006F8F10BD9C000020224BD3F8183123B1CE
:10263000204B0122C3F8242170471E4A0023C2F810
:102640002431D2F80C31B3FA83F3DBB2C3F11F03A8
:1026500003EB830081000A44126B42B94FF0500330
:1026600083F31188BFF36F8FBFF34F8FFEE7114ADB
:1026700003EB830081001144486B406848633032AB
:1026800003EB830C4FEA8C0108310A44904209D0D5
:10269000084903EB83039A000A44536BDB68C1F8D3
:1026A00000317047406862469100024A0A44506314
:1026B000EEE700BF9C000020064BD3F804313BB18D
:1026C000044BD3F818310BB100207047022070473B
:1026D000012070479C00002082B0002301930D4B25
:1026E0001B68B3F1FF3F08D04FF0500383F311880C
:1026F000BFF36F8FBFF34F8FFEE74FF0500383F3AD
:102700001188BFF36F8FBFF34F8F019B002BFCD05D
:1027100002B070470800002008480068006880F395
:1027200008884FF0000080F3148862B661B6BFF3EA
:102730004F8FBFF36F8F00DF00BF000008ED00E098
:10274000DFF80C00016841F470010160704700007F
:1027500088ED00E04FF0807340F8043C21F0010167
:1027600040F8081C054B40F80C3C40F8202C6FF05A
:10277000020340F8243C4438704700BFD9260008C3
:10278000074B19680868B0E8F04F80F30988BFF379
:102790006F8F4FF0000080F311887047AFF3008017
:1027A0009C0100204FF0500383F31188BFF36F8F1B
:1027B000BFF34F8F0B4A136801331360012B00D016
:1027C00070474FF0E023D3F8043D13F0FF0FF7D02C
:1027D0004FF0500383F31188BFF36F8FBFF34F8F18
:1027E000FEE700BF08000020094B1B6843B94FF00B
:1027F000500383F31188BFF36F8FBFF34F8FFEE752
:10280000013B034A13600BB983F31188704700BF83
:102810000800002000000000000000000000000090
:10282000EFF30980BFF36F8F154B1A681EF0100F7E
:1028300008BF20ED108A20E9F04F10602DE9090053
:102840004FF0500080F31188BFF34F8FBFF36F8FAD
:10285000FFF7EAFE4FF0000080F3118809BC196809
:102860000868B0E8F04F1EF0100F08BFB0EC108AF7
:1028700080F30988BFF36F8F704700BFAFF300800C
:102880009C01002008B54FF0500383F31188BFF37B
:102890006F8FBFF34F8FFFF74BFD28B14FF0E02351
:1028A0004FF08052C3F8042D002383F3118808BD34
:1028B0004FF0E022002313619361054B1B6805492B
:1028C000A1FB03139B09013B53610723136170476D
:1028D00028000020D34D62104FF0E023D3F8002DE4
:1028E0003D4B9A421BD04FF0E023D3F8002D3B4BD9
:1028F0009A421DD030B583B0394B1A78D2B20192CA
:10290000FF221A701B78DBB28DF803309DF803307C
:1029100003F05003334A1370072353601BE04FF05A
:10292000500383F31188BFF36F8FBFF34F8FFEE720
:102930004FF0500383F31188BFF36F8FBFF34F8FB6
:10294000FEE7284A5368013B53609DF803305B0063
:10295000DBB28DF803309DF8033013F0800FF0D117
:10296000204B5B68032B08D04FF0500383F3118892
:10297000BFF36F8FBFF34F8FFEE71B02194A5360FF
:1029800003F4E0635360019BDBB2154A13704FF010
:10299000E024D4F8203D43F47003C4F8203DD4F87B
:1029A000203D43F07043C4F8203DFFF781FF002530
:1029B0000D4B1D60FFF7C4FED4F8343F43F0404395
:1029C000C4F8343FFFF7A8FEFFF72EFEFFF784FEA2
:1029D000284603B030BD00BF71C20F4170C20F4125
:1029E00000E400E0C801002008000020104A12F0B6
:1029F000070F1AD0D11D21F00701C1F57053134400
:102A00000A460C490A60002048601344083B23F042
:102A100007038B6058601860981A50601360C86094
:102A200008614FF000434B6170474FF47053E8E783
:102A3000F0010020D0010020164B1A461B6883428B
:102A4000FBD3516802EB010C844509D0416800EBCF
:102A5000010C634509D00360904219D010607047A3
:102A60004068014451601046F0E710B4094CA46876
:102A7000A3420BD05B681944416013681B68036074
:102A8000904200D010605DF8044B70470460F7E797
:102A9000704700BFD001002038B50446FFF738FC6E
:102AA000374B9B68B3B1364B5B691C424ED1002C4F
:102AB0004ED004F1080214F0070F02D022F00702F2
:102AC0000832002A53D02E4B1B69934251D32C4914
:102AD0000C6804E0FFF78AFFE5E721461C466368BF
:102AE000934202D22368002BF7D1254B9B68A34267
:102AF00041D00D68083523680B6063689B1A102B62
:102B000010D9A01810F0070F08D04FF0500383F32E
:102B10001188BFF36F8FBFF34F8FFEE74360626092
:102B2000FFF78AFF6168164A13695B1A1361D2685E
:102B3000934201D2124AD360114B5A690A43626030
:102B4000002222609A6901329A6102E0002500E0C9
:102B50000025FFF779FC15F0070F0ED04FF050035A
:102B600083F31188BFF36F8FBFF34F8FFEE700250C
:102B7000EFE70025EDE70025EBE7284638BD00BF6D
:102B8000D001002098B338B50446A0F1080550F8EC
:102B9000043C174A5269134208D14FF0500383F3A3
:102BA0001188BFF36F8FBFF34F8FFEE750F8081CFB
:102BB00041B14FF0500383F31188BFF36F8FBFF320
:102BC0004F8FFEE723EA020340F8043CFFF7A0FB27
:102BD00054F8042C064C2369134423612846FFF75C
:102BE0002BFFE3690133E361FFF72EFC38BD70472B
:102BF000D001002008B50120FFF725F9FBE7000010
:102C0000034B036054330B6080231360704700BF95
:102C1000F03D002010B588B00DF1040C084C0FCC2D
:102C2000ACE80F0094E807008CE80700002101A839
:102C3000FFF7D6F8034BC3F8540208B010BD00BF2D
:102C4000BC7E0008F03D0020884202DB904202DC9E
:102C5000704708467047104670470000002113482F
:102C600032237F2921DC10B40BE001DB002212E0CB
:102C70004FF0FF320FE023230D4A535401317F29D7
:102C800010DC0C4C43F2390204FB0020020F073A1F
:102C9000002AEADD01221344222BECDD3A2BEBDD86
:102CA0003A23E9E75DF8044B7047704787D6120076
:102CB000484000206D4EC64110B5044608467D22AE
:102CC0000221FFF7C1FF064B1A5C033A04EB8401B3
:102CD00003EB8101C1F88000C1F8842010BD00BF62
:102CE00048400020084B93F8A82082F0010283F8A6
:102CF000A820002283F8A9200022C3F8AC20034BAF
:102D00004FF07E521A607047484000202400002097
:102D1000154BD3ED007A9FED157A67EE877A144B49
:102D200093ED2B7A77EE877AC3ED2B7AB7EE007AA4
:102D3000F4EEC77AF1EE10FA04DB83ED2B7A0A4B3E
:102D40000C4A1A600A4BD3ED2B7AF5EEC07AF1EEFD
:102D500010FA00D970470022C3F8AC20024B4FF0A4
:102D60007E521A60F6E700BF24000020295C0F3D68
:102D700048400020000080BF08B50A4A92F8B030F1
:102D800092F8B120934209D20233DBB2054981F8AF
:102D9000B0309A4201D281F8B02008BDFFF7A2FFFF
:102DA000FBE700BF484000200C4991F8A83003EB36
:102DB000830082000A4492F8902001320848A0FB68
:102DC00002C000F4FF7C0CEB5000121A03EB8303EB
:102DD0009800014481F89020704700BF48400020CF
:102DE000ABAAAAAA0C4991F8A83003EB8300820091
:102DF0000A4492F8902002320848A0FB02C000F476
:102E0000FF7C0CEB5000121A03EB83039800014483
:102E100081F89020704700BF48400020ABAAAAAAC2
:102E200008B5FE2000F0A4FE042821D0022821D0FD
:102E3000012821D0FD2000F09BFE04281ED002288E
:102E40001ED001281ED0FB2000F092FE04281BD0CB
:102E500002281BD001281BD0F72000F089FE04288F
:102E600018D0022819D0012819D06FF0630000E0B3
:102E7000012008BD0220FCE70320FAE70420F8E760
:102E80000520F6E70620F4E70720F2E70820F0E740
:102E90000920EEE74FF0FF30EBE70020E9E76FF0A5
:102EA0000100E6E770B52DED068B2D4C94F8A85087
:102EB000AE0005EB850304EB830393F89010294AD9
:102EC00002EB0112D2ED028AD2ED037A77EEE87AB4
:102ED00094ED2B7A67EE877A78EEA78AD3ED237A82
:102EE000F8EEE77A9FED207A67EE877A9FED1F7AFA
:102EF00087EE87AA93ED209AB8EEC99AB0EE4A0AF7
:102F000001F04EFEB0EE408AF1EE0C9A60EE297AA6
:102F100039EE279A84ED2D9A2E4404EB860696ED21
:102F2000219AB8EEC99AB0EE4A0A01F07DFE60EE31
:102F3000299A39EE699A84ED2E9A28EE288A84ED32
:102F40002F8A20EE680A84ED300A84F8C4500023EA
:102F5000C4F8C830022384F8A930BDEC068B70BDDC
:102F600048400020D87E0008DA0F49400000344372
:102F700038B5D0B103464B4A92F8A920042A3AD07A
:102F8000B0F1FF3F38D010F1020F3AD0002A40F0E4
:102F90008180444A92F8A800023B062B2BD8DFE838
:102FA00003F0352A576D622A4600FFF757FE3D4C65
:102FB0006423C4F88830C4F89C302D23C4F88C30C6
:102FC0008723C4F8A030002584F8905084F8A450DA
:102FD0000C212846FFF770FE73210120FFF76CFEDD
:102FE00084F8A85084F8A9500023C4F8AC302E4BC4
:102FF0004FF07E521A6038BD002AFCD1FFF7D4FE94
:10300000F9E7002AF7D1FFF7EDFEF4E700EB8003C4
:10301000244A02EB8302D2F88C300233C2F88C309F
:10302000B42BE8DD1346B422C3F88C20E3E700EBB1
:1030300080031C4A02EB8302D2F88C30023BC2F8B8
:103040008C30002BD7DA13460022C3F88C20D2E74D
:1030500000EB8002134B03EB8203D3F8801001399D
:10306000FFF72AFEC7E700EB80020E4B03EB82035B
:10307000D3F880100131FFF71FFEBCE7094B012296
:1030800083F8A9200022C3F8AC20074B4FF07E52F2
:103090001A60B0E7012AAED10528ACD1FFF702FFD4
:1030A000A9E700BF4840002024000020F8B50646EC
:1030B0000D467F220021401BFFF7C6FD04467F22FC
:1030C00000217019FFF7C0FD074602E0114A1355B1
:1030D0000134BC421CDCA31B05FB05F203FB03F31C
:1030E0009A42F5DBD31A00EE103AB8EEC00A01F0AE
:1030F00039FDDFED097A20EE270ABDEEC00A054B47
:103100001B5D10EE102A13443F2BDFDD3F23DDE76C
:10311000F8BD00BF48400020CDCC0C3F70B52DED70
:10312000028B06460D4608EE102A08EE903A00245F
:1031300002E000232EE00134012C3BDC04EB84038D
:103140001E4A02EB8302D2F880309B1BD2F8842007
:10315000521B02FB02F203FB032300EE103AB8EE0F
:10316000C00A01F0FFFCF8EE487AF4EEC07AF1EE06
:1031700010FAE0D4C0EE276AB7EE007A37EE667A2E
:10318000F8EE687A67EE877AFDEEE77A17EE903A06
:10319000002BCEDB04EB8402084901EB8201D1F85D
:1031A0008820D31AC1F88830002BC4DA0022C1F875
:1031B0008820C0E7BDEC028B70BD00BF48400020F6
:1031C000F8B50D461D4C94F8A83003EB830304EBCF
:1031D000830393F890707F220021FFF735FD0646A8
:1031E000C4F8CC003F2200212846FFF72DFDC4F88B
:1031F000D000012384F8B030114D05EB07152F796D
:1032000084F8B17039463046FFF750FF6B793A4683
:10321000D4F8D010D4F8CC00FFF780FFD4F8883071
:103220003BB1D4F89C3023B1044B032283F8A9208E
:1032300003E0024B042283F8A920F8BD4840002097
:10324000D87E000838B53E4BD3ED326A70EE266A60
:10325000C3ED326A93ED357A20EE077AD3ED2F7AFB
:1032600037EE277A83ED2F7ADFED367A60EE277A14
:1032700093ED306A77EE867AC3ED307A27EE007AE6
:1032800093ED2D6A37EE067A83ED2D7A67EE807A1C
:1032900093ED2E6A77EE867AC3ED2E7AB6EE006A4B
:1032A00037EE067ABDEEC77A17EE100A77EE867A09
:1032B000FDEEE77A17EE904A7F2809D8002C07DB4D
:1032C0003F2C05DC1E4B195CA14210DD002323E0DE
:1032D0007F220021FFF7B8FC05463F22002120464F
:1032E000FFF7B2FC01462846FFF76AFF38BDFFF73B
:1032F00067FFFBE703EB8302114901EB8201D1F881
:103300008020121AD1F88410091B01FB01F102FB85
:103310000212092A10DD0133012BE7DCDAB2084979
:1033200091F8C4108A42E5D1DFED077AF4EEE76A3E
:10333000F1EE10FADED5EEE72146FFF741FFD5E7C3
:10334000484000200000B4428FC2F53D7F2803D8DA
:10335000002901DB3F2900DD704708B5C9B2C0B2C2
:1033600000F084FD08BD000038B5002508E001220A
:1033700021462846FFF7EAFF01343F2CF7DD0135EF
:103380007F2D02DC014B5C5DF7E738BD4840002033
:103390002DE9F0478146884615461F46C2F1000ACE
:1033A000564613E00134AC420FDC06FB06FC04FB7E
:1033B00004CC05FB05F39C45F4DC3A4606EB08011A
:1033C00004EB0900FFF7C2FFECE70136AE4201DC77
:1033D0005446E8E7BDE8F0872DE9F04F83B0054695
:1033E0000E46914601939DF830A0824223DDA2EB68
:1033F0000008A94522DD01230093019BB34221DD92
:10340000F71A019BB34220DD4FF0010B08EB0704D4
:10341000524631462846FFF799FF4D4518D06300C4
:10342000B7EB440F02DC3C44009A15449845EFDBAF
:1034300044445E44ECE7A0EB0208DAE74FF0FF33C8
:103440000093DAE7019B9F1BDBE74FF0FF3BDDE7D3
:10345000019B9E42E3D103B0BDE8F08F10B52DED86
:10346000048B0446027C314B03EB021393ED028A7A
:10347000D3ED037A77EEC87A67EE807A38EE278A42
:10348000D0ED037AF8EEE77A9FED297A67EE877A36
:103490009FED287AC7EE878AB0EE680A01F080FBBC
:1034A00060EE089AB0EE680A01F0BEFB20EE489A82
:1034B000D4ED007AF8EEE78A94ED018AB8EEC88A76
:1034C000002400E001340D2C2CDCDFED1B7A29EE0A
:1034D000A77A78EE878A69EE277A38EE278ADFEDB9
:1034E000177A39EE279AF6EE007A38EEA77ABDEE13
:1034F000C77A17EE100A78EE277AFDEEE77A17EE14
:10350000901A7F280ED800290CDB3F290ADC0C4BCF
:103510001B5C8B4206DD14F0010FD3D10122FFF7B3
:1035200015FFCFE7BDEC048B10BD00BFD87E0008AF
:10353000DA0F4940000034438FC2753DCDCCAC401A
:10354000484000202DE9F04F85B007468B461546D0
:103550001C464FF0000A564604E0013D6B00C3F1E3
:1035600001039A44B54241DBEB1906EB0B092246F5
:10357000494601931846FFF7E9FEF31905EB0B08DE
:103580002246414602931846FFF7E0FEBA1B134657
:103590002246414603931846FFF7D8FEA7EB0508DD
:1035A000224649464046FFF7D1FEABEB06092246CC
:1035B00049464046FFF7CAFEABEB050822464146A6
:1035C0000398FFF7C3FE224641460298FFF7BEFE6E
:1035D000224649460198FFF7B9FE013673000133D0
:1035E0009A44AAEB0503002BB7DABBE705B0BDE8A8
:1035F000F08F38B504460D464AB101230222FFF789
:10360000C7FE0122E91E2046FFF7A0FE38BD0123B8
:103610000222FFF797FFF9E770B58AB0002108464C
:1036200000F0C4FC554DD5F88820554902A800F09B
:10363000F9FD544E012396E8060002A800F09EFC16
:103640000021402000F0B2FCD5F89C204E4902A891
:1036500000F0E8FD012396E8060002A800F08EFCC9
:1036600095F8A8400C21002000F0A0FC04EB840396
:1036700005EB830393F890201201D3F88C30434973
:103680008A58434902A800F0CDFD012396E80600C0
:1036900002A800F073FC95F8A930012B06D0374B37
:1036A00093F8A930042B3DD00AB070BD01240094DA
:1036B00038237C2219460420FFF78EFE00943E2317
:1036C0007C2219460420FFF787FE00943E23042243
:1036D00038211046FFF780FE00943E237C223821DB
:1036E0001046FFF779FED5ED2B7A9FED2A7A67EE2B
:1036F000877A76220021FDEEE77A17EE900AFFF72F
:10370000A3FA0646002509E0012204F13901681DEB
:10371000FFF71CFE0134042CF6DD0135B542BEDA9C
:103720000024F8E71E21142000F040FC134BD3F8CE
:1037300088301BB9114AD2F89C208AB1BBB9164A0D
:10374000012306CA154800F019FC3421062000F0B8
:103750002DFC0C4A012306CA114800F00FFCA3E718
:103760000D4A012306CA0F4800F008FCEDE70A4A9B
:10377000012306CA0C4800F001FCE6E7484000209F
:10378000347F00081C000020407F0008D87E00081D
:10379000487F00080000EC42140000205C7F000815
:1037A0006C7F0008547F0008647F00082DE9F04317
:1037B0002DED028B83B0002000F0B6FAFFF7D4FDA8
:1037C000564BD3F88000D3F8841093F8A83043B94F
:1037D000524B93F8A930042B01D0012202E00022C1
:1037E00000E00022FFF705FF4C4BD3F89400D3F81C
:1037F000981093F8A830012B1AD00022FFF7F9FE99
:10380000464B93F8A930012B1BD9444B93F8A930B0
:10381000022B61D0414B93F8A930032B73D0FFF7F3
:10382000FBFE00F091FA03B0BDEC028BBDE8F08323
:103830003A4B93F8A930042B01D00122DEE7002295
:10384000DCE7364E96F8A85006F18008AF0005EB8D
:10385000850308EB830806EB8303D3ED237AF8EEA8
:10386000E77A9FED2F7A67EE877A9FED2E7AC7EE83
:10387000878AD3F88090B0EE680A01F091F9B2EE31
:10388000048A20EE080ABDEEC00A10EE104A4C442D
:103890002F4406EB8707D7F88450B0EE680A01F092
:1038A000C3F920EE080ABDEEC00A0123009310EE12
:1038B000103AEB1A224629464846FFF78DFD96F846
:1038C000A930012B05D09FED180A4046FFF7C6FD31
:1038D0009BE796ED2B0AF8E7104BD3ED2D7AF6EE29
:1038E000006A77EEA67A93ED2E7A37EE267A0122D9
:1038F000BDEEC77A17EE101AFDEEE77A17EE900AC2
:10390000FFF724FD86E70548012390F8B020D0F8A2
:10391000D010D0F8CC00FFF715FE80E7484000201B
:10392000DA0F494000003443CDCC0C3F30B583B0B2
:10393000FEF7F8FC01906FF063050FE0124B93F86F
:10394000A930012B15D0022B16D0032B19D0FFF76D
:103950002DFF1E2101A8FEF7EFFD2546FFF760FAB7
:1039600004468542EAD010F1640FE7D0FFF700FB70
:10397000E4E7FFF7CDF9EAE79FED040AFFF762FC01
:10398000E5E7FFF7F9F9E2E7484000208FC2F53C90
:1039900030B583B0FFF762F9194C6423C4F888305E
:1039A000C4F89C302D23C4F88C308723C4F8A03091
:1039B000002584F8905084F8A4500C212846FFF785
:1039C0007BF973210120FFF777F984F8A85084F878
:1039D000A9500023C4F8AC300A4A4FF07E51116060
:1039E000C4F8D430FFF7E2FE0195022300932B4682
:1039F0004FF4007204490548FEF723FC03B030BDC4
:103A00004840002024000020787F00082D3900085D
:103A100084B000220092154B196B41F080011963AC
:103A2000196B01F08001009100990192196B41F02E
:103A300004011963196B01F00401019101990292CB
:103A4000196B41F001011963196B01F00101029139
:103A5000029903921A6B42F002021A631B6B03F085
:103A600002030393039B04B0704700BF0038024079
:103A700008B50B480B4B03600B4B4360002383607E
:103A8000C3604FF48042026143618361C36103629A
:103A9000FDF7DAF900B908BD00F0C4F8FBE700BF94
:103AA0002041002000540040A086010030B589B0BC
:103AB0000023039304930593069307930268154B21
:103AC0009A4201D009B030BD00250195124C236BFC
:103AD00043F002032363236B03F002030193019B72
:103AE0004FF440730393122304930123059303239C
:103AF00006930423079303A90848FCF725FE0295C3
:103B0000236C43F400132364236C03F40013029327
:103B1000029BD7E7005400400038024000040240F6
:103B200010B582B000238DF807300DF10702022195
:103B3000E22000F055FA68B900238DF807300DF146
:103B400007020121E22000F04BFA044638B9204672
:103B500002B010BD0446044800F05CFAF7E70348E1
:103B600000F058FAF3E700BF987F0008B07F000824
:103B700010B582B00446FFF7D3FF08BB8DF80740AD
:103B80000DF107020321E22000F02AFAE0B90DF15D
:103B90000701E22000F038FAD0B99DF8073003F0B1
:103BA0007000702833D013F0100F16D1A4F1F70273
:103BB000072A12D8DFE802F01011111110111010AD
:103BC000154800F027FAD9E7144800F023FADEE799
:103BD000134800F01FFAE0E7042013F0200F0AD189
:103BE000A4F1F702072A06D8DFE802F0040505056C
:103BF00004050404022013F0400F09D1F73C072C00
:103C000006D8DFE804F007050505070507070020CB
:103C100002B010BD0120FBE7C47F0008D87F000878
:103C2000EC7F000872B6FEE700B595B030220021A7
:103C300008A800F019FB002303930493059306934F
:103C400007930193214A116C41F080511164126C69
:103C500002F080520192019A02931D4B1A6842F4BD
:103C600080421A601B6803F480430293029B012385
:103C700008934FF48033099302230E934FF480028C
:103C80000F92192210924FF4A872119212930423EA
:103C9000139308A8FDF7E4FB98B90F2303930223BD
:103CA0000493002305934FF4A05306934FF48053DD
:103CB0000793052103A8FDF723FE20B915B05DF891
:103CC00004FBFFF7AFFFFFF7ADFF00BF0038024076
:103CD0000070004008B5FCF78DFCFFF7A5FFFFF76B
:103CE00097FEFFF7C5FE00F021FA00F055F8FFF748
:103CF0004FFEFEF78FFFFEF76EF8FEE700B587B0C8
:103D00008DF817000A230293012301930DF1170286
:103D10000092002278210348FDF774F907B05DF89E
:103D200004FB00BF20410020002303E0FF21054ADF
:103D3000D1540133B3F5806F03D20028F6D1014688
:103D4000F5E770477441002010B584B000241AE0F4
:103D5000A4F15000C0B2FFF7D1FF0020FFF7CEFF63
:103D60001020FFF7CBFF6423029380230193084BBD
:103D700003EBC41300930123402278210548FDF78B
:103D800041F90134E4B2072CE2D904B010BD00BF00
:103D9000744100202041002008B56420FCF756FC47
:103DA000AE20FFF7ABFF2020FFF7A8FF1020FFF7A2
:103DB000A5FFB020FFF7A2FFC820FFF79FFF00205C
:103DC000FFF79CFF1020FFF799FF4020FFF796FFB9
:103DD0008120FFF793FFFF20FFF790FFA120FFF75F
:103DE0008DFFA620FFF78AFFA820FFF787FF3F205F
:103DF000FFF784FFA420FFF781FFD320FFF77EFFAA
:103E00000020FFF77BFFD520FFF778FFF020FFF7BA
:103E100075FFD920FFF772FF2220FFF76FFFDA202E
:103E2000FFF76CFF1220FFF769FFDB20FFF766FF4B
:103E30002020FFF763FF8D20FFF760FF1420FFF7BE
:103E40005DFFAF20FFF75AFF0020FFF76DFFFFF780
:103E50007BFF054B0022A3F80024A3F802240120D5
:103E600083F8050408BD00BF7441002010F0800FE6
:103E700026D13F2924D810B4124B93F8043413B13F
:103E8000B2FA82F25209012A0FD0CB0800EBC3101C
:103E90000C4C225C01F0070101238B40DB435BB239
:103EA000134023545DF8044B7047CB0800EBC3105C
:103EB000044C235C01F007018A4013432354F1E7CB
:103EC000704700BF744100202DE9F04782B0814661
:103ED00002A800E906009846274BB3F800349DF885
:103EE000006033447F2B42DC234BB3F802349DF84F
:103EF00001A053443F2B3CDC002523E01E4BB3F8CC
:103F00000004B3F8021429442044B8FA88F2520994
:103F1000C9B2C0B2FFF7AAFF0134A64211D907FA0D
:103F200004F313F4004FE9D0134BB3F80004B3F8D3
:103F30000214294420444246C9B2C0B2FFF796FF9A
:103F4000EAE70135AA4508D9A9F1200303FB0A5382
:103F5000019A32F813700024DFE7074AB2F8003400
:103F60003344A2F80034484602B0BDE8F087002090
:103F7000FAE70020F8E700BF7441002030B583B0B5
:103F8000044602A800E906001D4600E0013420783E
:103F900048B12B4602AA12E90600FFF795FF024638
:103FA00020788242F2D003B030BD0000024BA3F86B
:103FB0000004A3F8021470477441002000B585B0D6
:103FC000642302930123019300920A4640EA03010D
:103FD0000248FDF7C9F805B05DF804FB2041002058
:103FE00000B585B020F00100642302930123019302
:103FF00000920A4601460348FDF704F805B05DF853
:1040000004FB00BF2041002008B50A460021FFF74D
:10401000D5FF08BD10B50446FCF7DAF84FF47A7303
:1040200082B221460148FDF76AFE10BD804500209E
:1040300000B583B0002200920D4B596C41F48041D1
:104040005964596C01F48041009100990192196CF6
:1040500041F0805119641B6C03F080530193019B64
:104060000F216FF00100FCF74BFB03B05DF804FB80
:10407000003802407047FEE7FEE7FEE7FEE77047C4
:1040800008B5FCF7D1FAFEF717FB012800D108BDEF
:10409000FEF7F8FBFBE7000010B503460C4A0D499C
:1040A0000D48006840B10C4800680344521A93421E
:1040B00006D8094A136010BD0748084C0460F2E7AF
:1040C00000F0DAF80C2303604FF0FF30F3E700BF95
:1040D00000000220000400007C4500201047002062
:1040E0000F49D1F8883043F47003C1F888300D4B84
:1040F0001A6842F001021A60002098601A6822F0E3
:10410000847222F480321A60074A5A601A6822F4D4
:1041100080221A60D8604FF000638B60704700BF48
:1041200000ED00E0003802401030002408B50A48D5
:104130000A4B03604FF4E133436000238360C360A4
:1041400003610C2242618361C361FDF7A8FD00B9E0
:1041500008BDFFF767FDFBE7804500200014014024
:1041600000B589B000230393049305930693079346
:104170000268154B9A4202D009B05DF804FB002199
:10418000019103F592335A6C42F020025A645A6C42
:1041900002F020020192019A02911A6B42F004028D
:1041A0001A631B6B03F004030293029BC023039367
:1041B00002230493032306930823079303A90348C8
:1041C000FCF7C2FAD8E700BF001401400008024023
:1041D000DFF834D0002103E00C4B5B58435004312E
:1041E0000B480C4B42189A42F6D30B4A02E00023CC
:1041F00042F8043B094B9A42F9D3FFF771FF00F0F4
:1042000041F8FFF767FD7047000002200C840008AA
:10421000000000207C0000207C00002010470020CF
:10422000FEE700000EB410B59DB01FAB02900690E3
:104230006FF000410A48079104910A4953F8042B92
:104240000591002402A9006801931B9400F0A2F9D3
:10425000029B1C701DB0BDE8104003B0704700BF4A
:104260002C0000200802FFFF02440346934200D1C5
:10427000704703F8011BF9E7014B1868704700BF4E
:104280002C00002070B50D4D0D4C641BA4100026B1
:10429000A64209D10B4D0C4C01F0FAF9641BA41095
:1042A0000026A64205D170BD55F8043B984701365B
:1042B000EEE755F8043B98470136F2E7048400081E
:1042C00004840008048400080884000870477047CC
:1042D0000A44914200F1FF3300D1704710B511F844
:1042E000014B03F8014F9142F9D110BD38B5054695
:1042F000002941D051F8043C0C1F002BB8BFE41832
:1043000000F0E0F81D4A136833B963601460284672
:10431000BDE8384000F0DCB8A34208D92068211875
:104320008B4201BF19685B6809182160EDE71A46E6
:104330005B680BB1A342FAD911685018A0420BD1A7
:1043400020680144501883421160E0D118685B680E
:10435000536008441060DAE702D90C232B60D6E7DB
:10436000206821188B4204BF19685B68636004BF32
:10437000091821605460CAE738BD00BF0C4700200F
:1043800070B50F4E0C463168054611B900F0A4FB1C
:1043900030602146284600F09FFB431C03D14FF0BC
:1043A000FF34204670BDC41C24F00304A042F8D0A2
:1043B000211A284600F090FB0130F2D1EFE700BF50
:1043C000084700202DE9F843CD1C25F003050835EA
:1043D0000C2D38BF0C25002D064601DBA94204D95F
:1043E0000C2333600020BDE8F883DFF8D48000F0B0
:1043F00069F8D8F800301C4644BB29463046FFF720
:10440000BFFF431C044658D1D8F800402746002F70
:1044100043D1002C4BD023683946304604EB0309C6
:1044200000F05AFB814542D121686D1A2946304679
:10443000FFF7A6FF01303AD023682B442360D8F859
:1044400000305A6862BBC8F800700FE02268521B47
:1044500020D40B2A17D96119A342256018BF5960CF
:10446000636808BFC8F8001062514B60304600F026
:104470002FF804F10B00231D20F00700C21A1CBF07
:104480001B1AA350AFE76268A3420CBFC8F8002014
:104490005A60EBE723466468AEE73C467F68B6E7C0
:1044A0001A465B68A342FBD100235360DEE70C236E
:1044B0003360304600F00CF894E70560D6E700BFA3
:1044C0000C4700200148FFF701BF00BF0447002050
:1044D0000148FFF7FCBE00BF044700202DE9F0476C
:1044E0008E681F46BE420B6882460C4690462DD809
:1044F000B1F90C2012F4906F26D06569096905EBBB
:104500004505A3EB010905EBD5757B1C4B446D10EC
:104510009D4238BF1D46530527D52946FFF752FF58
:10452000064660B321694A46FFF7D2FEA38923F409
:10453000906343F08003A381266165614E44A5EB3F
:1045400009052660A5603E46BE4200D93E46206869
:104550003246414600F0A6FAA3689B1BA36023687D
:10456000334423600020BDE8F0872A4600F0C4FAF7
:1045700006460028E0D121695046FFF7B7FE0C231C
:10458000CAF80030A38943F04003A3814FF0FF3005
:10459000E9E700002DE9F04F98468B891B069DB096
:1045A00007460D46144610D50B6973B94021FFF735
:1045B00009FF2860286130B90C233B604FF0FF30C1
:1045C0001DB0BDE8F08F40236B61002309932023C9
:1045D0008DF82930CDF80C803023DFF89C818DF8E0
:1045E0002A304FF0010923469A4613F8012B0AB1ED
:1045F000252AF9D1BAEB040B0BD05B46224629469B
:104600003846FFF76BFF013000F0A780099A5A4443
:1046100009929AF80030002B00F09F8000234FF0A1
:10462000FF32CDE905230AF1010A049307938DF8BF
:1046300053301A935446052214F8011B4E48FBF7D9
:10464000CFFD049AD8B9D00644BF20238DF853304B
:10465000110744BF2B238DF853309AF800302A2BD2
:1046600015D0079A544600204FF00A0C214611F845
:10467000013B303B092B4BD9B0B1079214E0A0EBC2
:10468000080309FA03F313430493A246D2E7039BFA
:10469000191D1B680391002BBBBF5B4242F0020255
:1046A00007930793B8BF049223782E2B0AD163781F
:1046B0002A2B32D1039B1A1D1B68039243EAE37332
:1046C00002340593DFF8C0A0217803225046FBF79F
:1046D00087FD38B1049BA0EB0A00402282401343BF
:1046E0000134049314F8011B24488DF82810062285
:1046F000FBF776FD002836D0214B1BBB039B07330D
:1047000023F0070308330393099B334409936AE7B3
:104710000CFB02320C460120A8E70023013405936C
:1047200019464FF00A0C204610F8012B303A092A9E
:1047300003D9002BC6D00591C4E70CFB0121044628
:104740000123F0E703AB00932A460E4B04A9384639
:10475000AFF30080421C0646D6D1AB895B063FF51D
:104760002DAF09982CE703AB00932A46054B04A90B
:10477000384600F079F8EDE7F87F0008028000087D
:1047800000000000DD440008FE7F00082DE9F0472E
:10479000164698468A680B69DDF820909342B8BFA8
:1047A0001346336091F8432007460C460AB10133A3
:1047B00033602368990642BF33680233336025684B
:1047C00015F0060506D104F1190AE36832689B1A50
:1047D000AB4226DC94F843302268003B18BF01232B
:1047E00092062BD404F1430241463846C8470130B3
:1047F0001ED02368226903F00603042B02BFE5687C
:104800003368ED1AA3680CBF25EAE57500259342CD
:10481000C4BF9B1AED1800261A34B5421AD10020E5
:1048200008E00123524641463846C847013003D1CB
:104830004FF0FF30BDE8F0870135C6E7E1185A1C9C
:10484000302081F84300224494F8451082F8431048
:104850000233C7E70123224641463846C8470130A4
:10486000E6D00136D9E700002DE9FF470F7E0C9E08
:10487000782F914680460C469A4601F1430207D8AC
:10488000622F0AD8002F00F0D180582F00F0B88096
:1048900004F1420684F842703AE0A7F16303152B55
:1048A000F6D801A151F823F0014900081549000884
:1048B0009148000891480008914800089148000874
:1048C00015490008914800089148000891480008DF
:1048D00091480008134A00083F490008CD490008E4
:1048E0009148000891480008354A0008914800089E
:1048F0003F4900089148000891480008D549000840
:1049000033681A1D1B68326004F1420684F8423095
:1049100001239CE033682068191D3160060601D52B
:104920001D6803E04506FBD5B3F90050002D03DAFE
:104930002D236D4284F8433058480A2311E0216842
:104940003368080653F8045B02D4490648BFADB289
:104950006F2F5248336014BF0A230823002184F8C4
:1049600043106668A660002E05DB21682E4321F007
:10497000040121604BD01646B5FBF3F103FB115740
:10498000C75D06F8017D2F46BB420D46F4D9082BC2
:104990000BD12368DF0708D5236961689942DEBF20
:1049A000302306F8013C06F1FF36921B2261CDF858
:1049B00000A04B4603AA21464046FFF7E7FE013020
:1049C0004AD14FF0FF3004B0BDE8F087236843F0D0
:1049D000200323603248782784F8457023683168C3
:1049E0001F0651F8045B02D45F0648BFADB23160C8
:1049F000D90744BF43F0200323601DB11023ADE766
:104A00002648E9E7236823F020032360F6E71646EB
:104A1000BDE7336825686169181D30602E061B6884
:104A200001D5196002E06806FBD5198000232361D7
:104A30001646BCE733681A1D32601E6862680021A2
:104A40003046FBF7CDFB08B1801B606063682361D3
:104A5000002384F84330AAE723693246494640469A
:104A6000D0470130ADD023689B0713D4E068039B87
:104A70009842B8BF1846A6E7012332464946404649
:104A8000D04701309DD00135E36803995B1AAB42F2
:104A9000F2DCEBE7002504F11906F5E709800008D0
:104AA0001A800008884210B501EB020402D9844242
:104AB000234607D8431EA14208D011F8012B03F862
:104AC000012FF8E7024401468A4200D110BD13F8D5
:104AD000014D02F8014DF7E738B5064D00230446B5
:104AE00008462B60FFF7D8FA431C02D12B6803B1AC
:104AF000236038BD004700202DE9F04107461446E9
:104B00000D4621B9BDE8F0411146FFF75BBC2AB95B
:104B1000FFF7ECFB25462846BDE8F08100F01AF8C7
:104B20008442064602D8B4EB500FF4D821463846EA
:104B3000FFF748FC804608B94546ECE7B4422246F8
:104B4000294628BF3246FFF7C3FB29463846FFF700
:104B5000CDFBF1E751F8043C181F002BBCBF0B58EC
:104B6000C018704708B52DED028BB0EE408A00F0FA
:104B7000A1F8B4EE488AF1EE10FA0CD6DFED078A00
:104B8000B4EEE88AF1EE10FA05D5FFF775FB88EE72
:104B9000A80A21230360BDEC028B08BD00000000C1
:104BA00010EE103A07B51E4A23F00043934206D890
:104BB000DFED1C0A03B05DF804EB00F07FB8B3F141
:104BC000FF4F04D330EE400A03B05DF804FB6846A3
:104BD00000F014F900F00300012809D0022810D0D9
:104BE000B0B9DDED010A9DED000A00F067F8EBE7D2
:104BF000DDED010A9DED000A00F0B8F8B1EE400AC3
:104C0000E2E7DDED010A9DED000A00F057F8F5E757
:104C1000DDED010A9DED000A012000F0A7F8D3E7C1
:104C2000D80F493F0000000010EE103A07B51F4AA8
:104C300023F00043934207D8DFED1D0A002003B0A4
:104C40005DF804EB00F092B8B3F1FF4F04D330EEFF
:104C5000400A03B05DF804FB684600F0CFF800F0AE
:104C6000030001280AD002280FD0C0B9DDED010AE7
:104C70009DED000A012000F079F8EAE7DDED010A78
:104C80009DED000A00F01AF8E3E7DDED010A9DED65
:104C9000000A012000F06AF8B1EE400AD9E7DDED24
:104CA000010A9DED000A00F009F8F5E7D80F493F29
:104CB00000000000B1EEC00A7047000010EE103A8C
:104CC00023F00043B3F1485FF0EE406AB7EE000A0C
:104CD00004D2FDEEE67A17EE902A42B326EEA67ACB
:104CE000DFED1A7A9FED1A6A1A4AA7EE276A9342F5
:104CF000DFED197AE6EE077A9FED186AA7EE876A6C
:104D0000DFED177AE6EE077A9FED166AA7EE876A5F
:104D100060EEE60A26EE076AF6EE007AE7EE060A8D
:104D200067EE277A04D877EEE07A30EE670A7047AC
:104D30000D4A93429ABF03F17F4307EE103AB5EE56
:104D4000027A30EE470A77EEC77AECE74ED747ADE6
:104D5000F6740F319999993E7CF293B4010DD037D6
:104D6000610BB6BAABAA2A3D0000483F10EE103ADC
:104D700023F00043B3F1485F04D2FDEEC07A17EE92
:104D8000903A5BB320EE007ADFED157A9FED156A5D
:104D9000A7EE276ADFED147AE6EE077A9FED136A35
:104DA000A7EE876ADFED127A60EE076AE6EE077A11
:104DB00030B99FED106AA7EE276AA6EE260A704763
:104DC00067EEE67AB6EE006AE0EE867AD7EE870AFC
:104DD000DFED097AE6EEA70A30EE600A704700BF01
:104DE000D3C92E2F342FD7B21BEF3836010D50B94F
:104DF0008988083CABAA2ABEABAA2A3EF0B510EEC1
:104E0000106A884B26F000459D4287B0044605D8BD
:104E1000002380ED000A4360002022E0824B9D4287
:104E20003AD826F00043002E9FED807A804A23F086
:104E30000F0318DD934270EE477A09BF9FED7D7A2C
:104E4000DFED7D6ADFED7D6A77EEC77A37EEE67AD1
:104E500077EEC77A80ED007A77EEE67AC0ED017AD8
:104E6000012007B0F0BD934270EE077A09BF9FEDB5
:104E7000717ADFED716ADFED716A77EE877A37EE6E
:104E8000A67A77EEC77A80ED007A77EEA67AC0ED43
:104E9000017A4FF0FF30E4E7694B9D4273D800F090
:104EA000DDF89FED687AF6EE007AE0EE077AFDEE27
:104EB000E77AB8EEE77A17EE900ADFED5C7AA7EEB4
:104EC000670A1F28DFED5C7A67EE277AB1EE476A42
:104ED00070EE676A16EE901A09DC5B4A471E26F0F0
:104EE000004352F8272023F0FF03934207D1C1F378
:104EF000C752C2EBD552082A4FEAE55314DC2160B1
:104F000094ED007A30EE470A002E30EE670A84ED09
:104F1000010AA6DAB1EE477AB1EE400A84ED007AD2
:104F200084ED010A40429CE7DFED425AF0EE406A10
:104F3000E6EE256A70EE667AE6EE257ADFED3F5AF8
:104F4000D7EE257A76EEE75A15EE902AC2F3C751CE
:104F50005B1A192B04DCC4ED005AB0EE660ACFE7E9
:104F6000DFED3A5AB0EE660AA6EE250A76EEC07A72
:104F7000DFED376AE6EE257AD7EE267A30EE677AED
:104F800084ED007ABCE7B5F1FF4F06D370EE407AAE
:104F9000C0ED017AC0ED007A3EE7EA15863AA5EB4E
:104FA000C25307EE903ABDEEE77ADFED2A6AB8EE1B
:104FB000C77A77EEC77A8DED037A67EEA67ABDEEF3
:104FC000E77AB8EEC77A77EEC77A8DED047A67EEA6
:104FD000A67AF5EE407AF1EE10FACDED057A1ED103
:104FE000B5EE407AF1EE10FA0CBF012302231A4904
:104FF00001910221009103A8214600F037F8002E0C
:10500000BFF62FAFD4ED007AF1EE677AC4ED007AE7
:10501000D4ED017AF1EE677AC4ED017A82E70323D9
:10502000E5E700BFD80F493FE3CB1640800FC93FEB
:10503000D00FC93F004435374344353708A3852E88
:10504000800F494384F9223F2C80000800A3852E5D
:1050500032318D2400008043AC80000810EE103AFD
:1050600023F0004300EE103A704700002DE9F04FA6
:105070002DED048BD9B090460190B64A669818F190
:10508000040F52F820A00F4603F1FF3B26DBB8F1D6
:10509000030248BF08F10402D210551C67999FED26
:1050A000B17AE800A2EB0B060290A8EBC5050AEB6B
:1050B0000B0C1CAC01EB860E0020604510DD1CA91A
:1050C00001EB83000DF588790026564524DCDDF8D8
:1050D00004E0DFEDA47A8446002416E00022DCE739
:1050E000C6425DBF5EF8201007EE901AF8EEE77A30
:1050F000F0EE477AE4EC017A0130DEE7FEEC016A7B
:105100003CED017AE6EE877A01345C45F6DDE9ECA8
:10511000017A01360430D8E708A901EB8A0104912D
:105120006799DFED8F8A9FED8D9A01EB82020392E2
:105130005446A200059258AA02EB840212ED140A0A
:1051400044A908AA01EB840094462646002E4CDCB4
:105150002846CDE9062300F0F1F9B0EE408AB4EE1E
:10516000000A28EE000A00F04FFAF2EE007AA0EEF4
:10517000678A002DDDE90623FDEEC87A17EE909AC6
:10518000F8EEE77A38EE678A41DD04F1FF3C08A9C2
:10519000C5F1080E51F82C6046FA0EF0814400FA71
:1051A0000EF0361AC5F1070041F82C600641002EBA
:1051B0003CDD4FF0000E09F101097046744568DCD2
:1051C000002D03DD012D74D0022D7DD0022E2DD1B6
:1051D000B7EE000A30EE488A40B32846069300F046
:1051E000ADF9069B38EE408A20E060EE287A013E59
:1051F000FDEEE77AF8EEE77AA7EEC90ABDEEC00A3F
:10520000ACEC010A30ED010A37EE800A9EE705D1C9
:10521000601E08A951F82060F611C8E7F6EE007A82
:10522000B4EEE78AF1EE10FA31DA0026B5EE408AE4
:10523000F1EE10FA40F09880601E002250454BDAE3
:10524000002A65D0013C08AB083D53F82430002B00
:10525000F8D02846B7EE000A00F070F9631C44AAA3
:105260009FED3F7A990002EB83022346002B80F2E8
:10527000A9802346002BC0F2C78044AA02EB830515
:10528000DFF8D4C0DFED377A0020E21AB1E0022661
:105290008FE752F8041B48B921B1C1F5807142F87B
:1052A000041C01210EF1010E084687E7C1F1FF0140
:1052B000F5E704F1FF3C08AA52F82C2002F07F0227
:1052C00008A941F82C2081E704F1FF3C08AA52F814
:1052D0002C2002F03F02F3E708A951F82010013812
:1052E0000A43ABE7013250F8046D002EFAD005995D
:1052F00001F5B0710DEB0100E6181CA904F1010CD9
:105300004C3801EB86062244624504DA144610E765
:1053100004980122E7E70399DDF804E051F82C1026
:10532000059107EE901AF8EEE77A0024E6EC017A90
:10533000DFED0C7AB1465C4504DDE0EC017A0CF15E
:10534000010CE1E7FEEC016A39ED017A0134E6EE89
:10535000877AF0E7F0830008C483000800008043E8
:105360000000803B00000000029BB0EE480AA3EB67
:10537000080000F0E3F81FED077AB4EEC70AF1EE7B
:1053800010FA19DB5FED0A7A60EE277A08AAFDEEC3
:10539000E77A0835F8EEE77AA7EEC70AFDEEE77A76
:1053A000BDEEC00A10EE103A42F8243017EE903AE3
:1053B000013442F824304CE7BDEEC00A08AA10EED2
:1053C000103AF6E708A850F82300019007EE900A7B
:1053D000F8EEE77A013B67EE807A20EE070A62ED8D
:1053E000017A43E7FCEC016AB5EC017AE6EE877AD4
:1053F0000130504501DC9042F4DD58A800EB8202F8
:1054000042ED287A013B35E7669B022B09DC002B35
:1054100027DC40D009F0070059B0BDEC048BBDE893
:10542000F08F669B032BF5D130AA0B1F13441A464D
:105430002046002850DC2246012A5DDC30AB5FEDBF
:10544000377A0B44012C67DCDDED306A9DED317A53
:10545000002E67D1C7ED006A87ED017AC7ED027AA9
:10546000D8E730AB1FED417A0B442246002A24DAFC
:105470004EB3F1EE477AC7ED007ADDED307A77EE84
:10548000C77A31AA01239C4220DA0EB1F1EE677A85
:10549000C7ED017ABEE730AB5FED4E7A0B44002CCE
:1054A00005DA0EB1F1EE677AC7ED007AB2E733EDB7
:1054B000017A013C77EE877AF1E773ED017A013AE0
:1054C00037EE277AD2E7F0EE477AD4E7B2EC017AEA
:1054D000013377EE877AD6E772ED017AD2ED016A71
:1054E00037EEA67A013877EEC77A82ED007A77EE4A
:1054F000A67AC2ED017A9CE773ED017AD3ED016AD9
:1055000037EEA67A013A77EEC77A83ED007A77EE26
:10551000A67AC3ED017A8FE733ED017A013C77EE8D
:10552000877A8FE7F1EE666AB1EE477AC7ED006AD7
:1055300087ED017AF1EE677A90E700BF10EE103A3E
:1055400033F000422BD0B2F1FF4F02D330EE000A0D
:10555000704713F0FF4F23D1244BDFED257A98429B
:1055600020EE270A17DB10EE103AC3F3C752193AA0
:105570004CF25031884215DDDFED1E7ADFED1E6AF8
:1055800010EE103AB0EE677A002BB8BFF0EE667AF4
:1055900027EE870A7047DFED197A27EE800A7047F9
:1055A000D20DE5E71044FE28E6DC002806DD23F0F6
:1055B000FF4343EAC05300EE103A704710F1160F54
:1055C00009DADFED0E7ADFED0E6A10EE103AB0EE7A
:1055D000677A002BD9E7193023F0FF4343EAC05321
:1055E0009FED080A07EE903AD7E700BFB03CFFFFF7
:1055F0000000004CCAF24971CAF249F16042A20DA2
:105600006042A28D0000003310EE103AC3F3C7527F
:105610007F3A162A23F000412BDC002A12DADFED54
:10562000197A30EE270AB5EEC00AF1EE10FA06DD5F
:10563000002B24DA0029144B08BF4FF0004300EE82
:10564000103A7047114911410B42FAD0DFED0D7A43
:1056500030EE270AB5EEC00AF1EE10FAEFDD002BAE
:10566000BEBF4FF4000040FA02F29B1823EA010388
:10567000E5E7B1F1FF4FE4D330EE000A70470023B5
:10568000DDE700BFCAF24971000080BFFFFF7F0065
:10569000F8B500BFF8BC08BC9E467047F8B500BF1F
:0856A000F8BC08BC9E467047EF
:1056A80000000000000000000000000000000000F2
:1056B80000000000000000000000000000000000E2
:1056C80000000000000000000000000000000000D2
:1056D80000000000E003E003E003E003E003E00370
:1056E800E003E003C003C003C001C001C001C00162
:1056F800C001000000000000E003E003E003000038
:1057080000000000000000003C1E3C1E3C1E3C1E29
:105718003C1E3C1E3C1E0000000000000000000073
:105728000000000000000000000000000000000071
:10573800000000000000000000000000CE01CE03C1
:10574800DE039E039C039C07FF3FFF7F3807380F4B
:10575800780F780F780EFFFFFFFFF01EF01CE01C9B
:10576800E03CE03DE03900000000000000000000DF
:10577800FC03FE0FEE1FE01EE01EE01EE01EE01F11
:10578800E00FE007F003FC01FE01FE01FE01FE014F
:10579800FE01FE01FE3DFC3FF00FE001E0010000CC
:1057A80000000000033E07F78FE78EE79EE3BCE3A7
:1057B800B8E7F8E7F0F7E03FC001FF03FF07F3079A
:1057C800F30FF31EF33CF338F3787FF03FE000006B
:1057D8000000000000000000E007F80F780F781FB5
:1057E800781F781F780FF00FE00F801FC37FC3FB6F
:1057F800E7F3F7F1F7F0FFF07FF03EF87F7CFF3F2B
:10580800EF1F00000000000000000000E003E003BC
:10581800E003E003E003C003C00100000000000053
:105828000000000000000000000000000000000070
:105838000000000000000000000000000000000060
:105848003F007C00F001E001C003C007800780072B
:10585800800F000F000F000F000F000F000F800FC8
:1058680080078007C007C003E001F0017C003F000B
:105878000F000000007E001FC007C003E001F00118
:10588800F000F000F80078007800780078007800E0
:105898007800F800F000F000F001E001C003C00754
:1058A800001F007E00780000E003C003C001CE396D
:1058B800FF3F7F3F20037003F807780F3C1F38062F
:1058C80000000000000000000000000000000000D0
:1058D80000000000000000000000000000000000C0
:1058E8000000000000000000C001C001C001C001AC
:1058F800C001C001C001FFFFFFFFC001C001C0011E
:10590800C001C001C001000000000000000000004C
:10591800000000000000000000000000000000007F
:10592800000000000000000000000000000000006F
:105938000000E003E003E003E003E001E001E00130
:10594800C00180030000000000000000000000000B
:1059580000000000000000000000FE3FFE3F0000C5
:10596800000000000000000000000000000000002F
:10597800000000000000000000000000000000001F
:10598800000000000000000000000000000000000F
:1059980000000000000000000000E003E003E00356
:1059A800E003000000000000000000000F000F00EE
:1059B8001E001E003C003C0078007800F000F0005B
:1059C800E001E001C003C00380078007000F000F5B
:1059D800001E001E003C003C0078007800F000002B
:1059E800F007F80F7C1F3E3E1E3C1F7C1F7C0F7883
:1059F8000F780F780F780F780F780F781F7C1F7C3F
:105A08001E3C3E3E7C1FF80FF0070000000000001F
:105A180000000000F000F007F03FF03FF001F00157
:105A2800F001F001F001F001F001F001F001F001E6
:105A3800F001F001F001F001F001FF3FFF3F00002D
:105A48000000000000000000E00FF83F7C3C3C0034
:105A58003E003E003E003C003C007C00F800F001A7
:105A6800E003C0078007000F001E003E003CFE3F19
:105A7800FE3F00000000000000000000F00FF81FCB
:105A88007C1C3E003E003E003C003C00F800F00F4D
:105A9800F80F7C003E001E001E001E001E003E0087
:105AA8007C1CF81FE01F0000000000000000000040
:105AB8007800F800F800F801F803F807F807780FFD
:105AC800781E781E783C78787878FFFFFFFF78009A
:105AD8007800780078007800780000000000000066
:105AE80000000000FC1FFC1FFC1F001E001E001E03
:105AF800001E001EE01FF81FFC007C003E003E0058
:105B08001E003E003E003C007C1CF81FE01F000009
:105B18000000000000000000FC01FE078E0F001FBF
:105B2800001E003E003C003CF83DFC3F3E7F1F7ECF
:105B38000F3C0F3C0F3C0F3C0F3E1F1E3E1FFC0F3F
:105B4800F00300000000000000000000FF3FFF3FDE
:105B5800FF3F0F001E001E003C0038007800F000D8
:105B6800F000E001E001C003C0038007800F800F50
:105B7800000F001F001F00000000000000000000D0
:105B8800F807FC0F3E1F1E1E1E3E1E3E1E1E3C1F1B
:105B9800F80FF007F80FFC1E3E3E1F3C1F7C0F7CE1
:105BA8000F7C1F3C3E3FFC1FF00700000000000078
:105BB80000000000F007F80F7C1E3E3C1E3C1F7CD6
:105BC8001F7C1F7C1F7C1F3C3F3EFF1FEF071F00F1
:105BD8001E001E003E003C00F838F03FE01F0000A9
:105BE80000000000000000000000000000000000AD
:105BF80000000000E003E003E003E0030000000011
:105C080000000000000000000000E003E003E003E3
:105C1800E003000000000000000000000000000099
:105C28000000000000000000E003E003E003E003E0
:105C38000000000000000000000000000000E00379
:105C4800E003E003E003E001E001E001C0038003BA
:105C580000000000000000000000000003000F002A
:105C68003F00FC00F003C00F003F00FE003FC00FE4
:105C7800F003FC003F000F000300000000000000DC
:105C8800000000000000000000000000000000000C
:105C98000000000000000000FFFFFFFF0000000000
:105CA8000000FFFFFFFF00000000000000000000F0
:105CB80000000000000000000000000000000000DC
:105CC8000000000000E000F8007E801FE007F801F7
:105CD8007E001F007E00F801E007801F007E00F8AC
:105CE80000E000000000000000000000F01FFC3F82
:105CF8003E381F381F381E001E003C007800F00098
:105D0800E001C003C003C007C00700000000000096
:105D1800C007C007C0070000000000000000000026
:105D2800F803FE0F1E1F0F3E7F3CFF78EF79C77305
:105D3800C7F38FF38FF38FF39FF39FF3FF73FF7B0B
:105D4800F779003C1C1FFC0FF8030000000000005E
:105D580000000000000000000000E003E003F0077E
:105D6800F007F007780F780F7C0E3C1E3C1E3E3C77
:105D7800FE3FFF3F1F780F780FF007F007F0000095
:105D88000000000000000000000000000000F83FD4
:105D9800FC3F3E3C1E3C1E3C1E3C3E3C7C3CF03FD7
:105DA800F83F7E3C1F3C1F3C0F3C0F3C1F3CFE3F16
:105DB800F83F0000000000000000000000000000A4
:105DC8000000FF01FF07871F003E003C007C0078B1
:105DD8000078007800780078007C007C003E003F66
:105DE800831FFF07FF010000000000000000000003
:105DF800000000000000F07FFC7F7E781F781F788D
:105E08000F780F780F780F780F780F780F780F7852
:105E18001F781E787E78F87FE07F00000000000081
:105E280000000000000000000000FF3FFF3F003EB0
:105E3800003E003E003E003E003EFE3FFE3F003E6C
:105E4800003E003E003E003E003EFF3FFF3F000098
:105E58000000000000000000000000000000FF1F1C
:105E6800FF1F001E001E001E001E001E001EFF1F3A
:105E7800FF1F001E001E001E001E001E001E001E2A
:105E8800001E0000000000000000000000000000EC
:105E98000000FE03FF0F871F003E007C007C007897
:105EA80000F800F87FF87FF80F780F7C0F7C0F3E22
:105EB8008F1FFF0FFE03000000000000000000001D
:105EC8000000000000001F7C1F7C1F7C1F7C1F7CC3
:105ED8001F7C1F7C1F7CFF7FFF7F1F7C1F7C1F7C1C
:105EE8001F7C1F7C1F7C1F7C1F7C000000000000A3
:105EF80000000000000000000000FF3FFF3FE0033B
:105F0800E003E003E003E003E003E003E003E00371
:105F1800E003E003E003E003E003FF3FFF3F00008E
:105F28000000000000000000000000000000FC1F4E
:105F3800FC1F7C007C007C007C007C007C007C00DA
:105F48007C007C007C007C0078007800F838F03F0A
:105F5800C03F00000000000000000000000000003A
:105F680000001F3C1E3C3C3C783CF03CE03DE03FE0
:105F7800C03F803FC03FE03FF03DF03C783C7C3C78
:105F88003E3C1F3C0F3C00000000000000000000E9
:105F9800000000000000003E003E003E003E003EC3
:105FA800003E003E003E003E003E003E003E003EF9
:105FB800003E003E003EFF3FFF3F000000000000A3
:105FC800000000000000000000001FF81FFC1FFC7C
:105FD8003FFE3FFE3FFE7FFF77FF77FFF7F7E7F7CC
:105FE800E7F3E7F3C7F307F007F007F007F000005F
:105FF80000000000000000000000000000000F7C0E
:106008000F7C0F7E0F7F0F7F8F7F8F7FCF7FEF7B80
:10601800EF79FF79FF78FF787F783F783F781F78AE
:106028001F780000000000000000000000000000D1
:106038000000F007FC1F3E3E1F7C0F780F780FF81A
:106048000FF80FF80FF80FF80FF80F780F781F7C7C
:106058003E3EFC1FF00700000000000000000000AA
:10606800000000000000FC3FFF3F1F3E0F3E0F3EB8
:106078000F3E0F3E1F3E3F3EFC3FF03F003E003EBE
:10608800003E003E003E003E003E000000000000D2
:1060980000000000000000000000F007FC1F3E3E6A
:1060A8001F7C0F780F780FF80FF80FF80FF80FF81C
:1060B8000FF80F780F781F7C3E3EFC1FF8077C0016
:1060C8003F000F0003000000000000000000F03F48
:1060D800FC3F7E3C3E3C1E3C1E3C3E3C3C3CFC3C6B
:1060E800F03FE03FF03DF83C7C3C3E3C1E3C1F3C12
:1060F8000F3C00000000000000000000000000004D
:106108000000FC07FE1F0E3E003C003C003C003E29
:10611800C01FF80FFE037F001F000F000F001F2095
:106128003E3CFC3FF01F00000000000000000000A3
:10613800000000000000FFFFFFFFE003E003E003B2
:10614800E003E003E003E003E003E003E003E0032F
:10615800E003E003E003E003E003000000000000C8
:10616800000000000000000000000F7C0F7C0F7C86
:106178000F7C0F7C0F7C0F7C0F7C0F7C0F7C0F7CBF
:106188000F7C0F7C1E3C1E3C3E3EFC1FF0070000AF
:10619800000000000000000000000000000007F000
:1061A80007F007F80F780F7C1E3C1E3C1E3E3C1E75
:1061B8003C1F781F780FF80FF007F007F007E0038F
:1061C800E0030000000000000000000000000000E4
:1061D800000003E003F003F007F0E7F3E7F3E7F369
:1061E800E773F77BF77FFF7F7F7F7F7F7E7F7E3F31
:1061F8003E3E3E3E3E3E0000000000000000000023
:1062080000000000000007F80F7C1E3E3E3E3C1FC9
:10621800F80FF007E007E003E003F007F80F7C0F42
:106228007C1E3E3C1F780F780FF000000000000035
:106238000000000000000000000007F807780F7C4D
:106248001E3C1E3E3C1F780FF80FF007E003E003EA
:10625800E003E003E003E003E003E003E003000001
:106268000000000000000000000000000000FF7FA8
:10627800FF7F0F001F003E007C00F800F000E001E7
:10628800E003C007800F000F001E003E007CFF7F68
:10629800FF7F00000000000000000000FF078007EB
:1062A80080078007800780078007800780078007AE
:1062B800800780078007800780078007800780079E
:1062C80080078007800780078007FF07FF07000017
:1062D80000780078003C003C001E001E000F000FF4
:1062E80080078007C003C003E001E001F000F00070
:1062F800780078003C003C001E001E000F000F00D4
:1063080007000000F07FF000F000F000F000F0005F
:10631800F000F000F000F000F000F000F000F000F5
:10632800F000F000F000F000F000F000F000F000E5
:10633800F000F07FF07F0000C000C001C001E00362
:10634800E003F007F0077807780F380F3C1E3C1E73
:106358001E3C1E3C0F380F78077800000000000034
:106368000000000000000000000000000000000025
:106378000000000000000000000000000000000015
:106388000000000000000000000000000000000005
:10639800000000000000FFFFFFFF000000000000F9
:1063A800F0000000000000000000000000000000F5
:1063B80000000000000000000000000000000000D5
:1063C80000000000000000000000000000000000C5
:1063D80000000000000000000000000000000000B5
:1063E800F80FFC3F7C3C3E003E003E00FE07FE1FCF
:1063F8003E3E3E7C3E783E7C7E7CFF3FCF1F0000C9
:106408000000000000000000003C003C003C003C94
:10641800003C003CF83DFE3F3E3F1F3E0F3C0F3C1A
:106428000F3C0F3C0F3C0F3C1F3C1E3C3E3FFC3FCB
:10643800F03B000000000000000000000000000029
:106448000000000000000000FE03FF0F871F003E51
:10645800003E003C007C007C007C003C003E003E8E
:10646800871FFF0FFE03000000000000000000006F
:106478001F001F001F001F001F001F00FF07FF1F36
:106488003F3E1F3C1F7C1F7C1F7C1F781F781F7C92
:106498001F7C3F3C7F3EFF1FDF0F00000000000015
:1064A80000000000000000000000000000000000E4
:1064B800F803FC0F3E1F1E3E1F3C1F7CFF7FFF7F23
:1064C800007C007C003C003E071FFF0FFE0300001D
:1064D8000000000000000000FF01E103C003C00746
:1064E800C007C007FF7FFF7FC007C007C007C007FE
:1064F800C007C007C007C007C007C007C007C0075C
:10650800C0070000000000000000000000000000BC
:106518000000000000000000EF07FF1F7F3E1F3C47
:106528001F7C1F7C1F781F781F781F7C1F7C3F3CB7
:106538007F3EFF1FDF0F1E001E001E007C38F83F45
:10654800003C003C003C003C003C003CFC3DFE3F65
:106558009E3F1F3F1F3E1F3C1F3C1F3C1F3C1F3CD4
:106568001F3C1F3C1F3C1F3C1F3C0000000000005C
:1065780000000000F001F001000000000000000031
:10658800E07FE07FE001E001E001E001E001E001FF
:10659800E001E001E001E001E001E001E0010000CC
:1065A8000000000000000000F800F80000000000F3
:1065B80000000000F83FF83FF800F800F800F80085
:1065C800F800F800F800F800F800F800F800F80003
:1065D800F800F800F800F000F071E07F003C003CA3
:1065E800003C003C003C003C1F3C3E3C7C3CF83CF2
:1065F800F03DE03DC03FC03FE03FF03DF83C7C3C13
:106608003E3C1F3C1F3C0000000000000000000052
:10661800F07FF001F001F001F001F001F001F0016C
:10662800F001F001F001F001F001F001F001F001DA
:10663800F001F001F001F001F0010000000000009D
:106648000000000000000000000000000000000042
:106658009EF7FFFFFFFFFFFFE7FBE7F9C7F1C7F171
:10666800C7F1C7F1C7F1C7F1C7F1C7F1C7F100001A
:106678000000000000000000000000000000000012
:1066880000000000FC3DFE3F9E3F1F3F1F3E1F3C99
:106698001F3C1F3C1F3C1F3C1F3C1F3C1F3C1F3C1A
:1066A8001F3C000000000000000000000000000087
:1066B8000000000000000000F007FC1F3E3E1F3CE9
:1066C8001F7C0F780F780F780F780F781F7C1F3C8E
:1066D8003E3EFC1FF0070000000000000000000024
:1066E800000000000000000000000000F83DFE3F30
:1066F8003E3F1F3E0F3C0F3C0F3C0F3C0F3C0F3CF6
:106708001F3C1E3E3E3FFC3FF83F003C003C003C27
:10671800003C003C000000000000000000000000F9
:10672800EE07FE1F7E3E1E3C1E7C1E781E781E78DD
:106738001E781E781E7C3E7C7E3EFE1FDE0F1E00ED
:106748001E001E001E001E000000000000000000C9
:10675800000000007F1FFF1FE71FC71F871F001FC4
:10676800001F001F001F001F001F001F001F001F29
:10677800001F0000000000000000000000000000F2
:106788000000000000000000FC07FE1F0E1E003E77
:10679800003E003FE01FFC07FE003E001E001E00FA
:1067A8003E3CFC3FF01F000000000000000000001D
:1067B800000000000000800780078007FF7FFF7F40
:1067C8008007800780078007800780078007800789
:1067D80080078007C007FF03FF01000000000000DA
:1067E80000000000000000000000000000000000A1
:1067F8001E3C1E3C1E3C1E3C1E3C1E3C1E3C1E3CC1
:106808001E3C1E3C3E3C7E3CFE3EFE1FDE0F000052
:106818000000000000000000000000000000000070
:106828000000000007F00F780F781E3C1E3C1E3E4B
:106838003C1E3C1E780F780FF00FF007F007E003BE
:10684800E00300000000000000000000000000005D
:10685800000000000000000003F0E3F1E3F3E7F3B9
:10686800F7F3F7F3F77F777F7F7F7F7F7F7F3E3E6A
:106878003E3E3E3E3E3E000000000000000000009C
:106888000000000000000000000000000F7C1E3E19
:106898003C3E3C1FF80FF007F007E003F007F8074D
:1068A800F80F7C1E3E3E1F3C1F78000000000000D1
:1068B80000000000000000000000000000000000D0
:1068C80007F80F780F7C1E3C1E3C3C1E3C1E3C1FEC
:1068D800780FF80FF007F007E003E003C003C003E8
:1068E800C0038007800F007F000000000000000048
:1068F80000000000FF3FFF3F1F003E007C00F80043
:10690800F001E003C007800F001F001E003CFF7F5E
:10691800FF7F00000000000000000000FE01E0030F
:10692800C003C003C003C003E001E001E001C001EF
:10693800C003803F803FC003C001E001E001E001E7
:10694800C003C003C003C003E003FE017E000000D3
:10695800C001C001C001C001C001C001C001C00127
:10696800C001C001C001C001C001C001C001C00117
:10697800C001C001C001C001C001C001C001C00107
:10698800C0010000C03FE003E001E001E001E001D8
:10699800C001C003C003C001E001FE00FE00E00129
:1069A800C001C003C003C001E001E001E001E00153
:1069B800E003C03F003F00000000000000000000AE
:1069C8000000000000000000000000000000073F79
:1069D800C77FE773FFF17EF00000000000000000B1
:1069E800000000000000000000000000000000009F
:1069F800000000000000000000000000000000008F
:106A0800000000000000000000000000000000007E
:106A18000000000C000C000C000C000C000C000C1A
:106A2800000C000C000C000C0000000C000C000016
:106A3800000000000000001B001B001B001B001BC7
:106A4800000000000000000000000000000000003E
:106A58000000000000000000000080198019801963
:106A68008019C07FC07F80190033C07FC07F00338A
:106A78000033003300330000000000000000001E57
:106A8800003F807580650074003C001E000780058B
:106A9800806580658075003F001E000400040000CA
:106AA8000000007000D840D8C0D880D90073000614
:106AB800000C801BC036C066C046C00680030000BC
:106AC800000000000000001E003F003300330033C8
:106AD800001E000CC03CC066806380618063C03EBD
:106AE800801C0000000000000000000C000C000CDE
:106AF800000C000C00000000000000000000000076
:106B080000000000000000000000000080000001FC
:106B18000003000600060004000C000C000C000C2A
:106B2800000C000C000400060006000300018000B1
:106B3800002000100018000C000C000400060006DD
:106B480000060006000600060004000C000C0018F1
:106B5800001000200000000C002D003F001E003334
:106B6800000000000000000000000000000000001D
:106B78000000000000000000000000000000000C01
:106B8800000C000C000CC0FFC0FF000C000C000C37
:106B9800000C0000000000000000000000000000E1
:106BA80000000000000000000000000000000000DD
:106BB800000000000000000C000C000400040008A5
:106BC80000000000000000000000000000000000BD
:106BD8000000001E001E0000000000000000000071
:106BE800000000000000000000000000000000009D
:106BF8000000000000000000000000000000000C81
:106C0800000C000000000000000000030003000367
:106C18000006000600060006000C000C000C000C24
:106C28000018001800180000000000000000001EF6
:106C3800003F0033806180618061806D806D80617C
:106C4800806180610033003F001E000000000000EA
:106C580000000006000E001E003600260006000692
:106C680000060006000600060006000600060000F2
:106C7800000000000000001E003F807380618061FA
:106C8800800100030006000C001800300060807FBF
:106C9800807F0000000000000000001C003E006330
:106CA80000630003000E000E000380018001806174
:106CB8008073003F001E0000000000000000000676
:106CC800000E000E001E001E00160036003600667C
:106CD800807F807F0006000600060000000000009C
:106CE8000000007F007F006000600060006E007F91
:106CF80080638001800180618073003F001E000076
:106D0800000000000000001E003F8033806100602A
:106D1800006E007F80738061806180618033003FF6
:106D2800001E0000000000000000807F807F8001BE
:106D38000003000300060006000C000C000C00080D
:106D48000018001800180000000000000000001ED5
:106D5800003F8063806180610021001E003F8061E8
:106D6800806180618061003F001E0000000000001B
:106D78000000001E003F00738061806180618073A5
:106D8800803F801D800180610073003F001E00006D
:106D98000000000000000000000000000000000CDF
:106DA800000C000000000000000000000000000CC3
:106DB800000C0000000000000000000000000000BF
:106DC80000000000000C000C0000000000000000A3
:106DD8000000000C000C0004000400080000000083
:106DE8000000000080008003000E003800600038BA
:106DF800000E80038000000000000000000000007A
:106E080000000000000000000000807F807F00007C
:106E18000000807F807F000000000000000000006C
:106E280000000000000000000000000000400070AA
:106E3800001C000780010007001C007000400000D3
:106E480000000000000000000000001F803FC0712B
:106E5800C060C000C00180030007000E000C000CD9
:106E68000000000C000C0000000000000000001EE4
:106E7800003F803180718063806F806D806D806F8E
:106E8800806700600032003E001C00000000000027
:106E98000000000E000E001B001B001B001B8031B1
:106EA8008031803F803F8031C060C060C06000009A
:106EB800000000000000007C007E006300630063A7
:106EC8000063007E007E0063806180618063007FD4
:106ED800007E0000000000000000001E003F80311E
:106EE8008061006000600060006000600060806198
:106EF8008031003F001E0000000000000000007C00
:106F0800007F00638063806180618061806180614F
:106F1800806100630063007E007C000000000000C8
:106F28000000807F807F0060006000600060007F5C
:106F3800007F0060006000600060807F807F00004C
:106F4800000000000000807F807F0060006000601B
:106F58000060007F007F00600060006000600060EB
:106F680000600000000000000000001E003F8031AB
:106F78008061006000600060806380638061806180
:106F88008031803F001E000000000000000080618A
:106F980080618061806180618061807F807F8061A5
:106FA8008061806180618061806100000000000074
:106FB8000000003F003F000C000C000C000C000C0F
:106FC800000C000C000C000C000C003F003F0000FF
:106FD8000000000000008001800180018001800124
:106FE8008001800180018001806180618073003FA1
:106FF800001E0000000000000000C0608061006307
:1070080000660066006C0078007C0066006600631D
:1070180080618061C0600000000000000000006026
:107028000060006000600060006000600060006058
:10703800006000600060807F807F0000000000002A
:107048000000C071C071C07BC07AC06AC06AC06EDF
:10705800C064C060C060C060C060C060C060000044
:10706800000000000000807180718079807980794B
:10707800806D806D806D80658067806780678063C4
:1070880080630000000000000000001E003F003385
:1070980080618061806180618061806180618061E0
:1070A8000033003F001E0000000000000000007ECA
:1070B800007F80638061806180618063007F007EE3
:1070C80000600060006000600060000000000000D8
:1070D8000000001E003F0033806180618061806194
:1070E80080618061806580670033803F401E0000BA
:1070F800000000000000007E007F806380618061E6
:107108008063007F007E00660063006380618061A9
:10711800C0600000000000000000000E001F803169
:10712800803100300038001E0007800380618061D4
:107138008031003F001E0000000000000000C0FF7A
:10714800C0FF000C000C000C000C000C000C000C24
:10715800000C000C000C000C000C000000000000EB
:1071680000008061806180618061806180618061F0
:1071780080618061806180618073003F001E000033
:10718800000000000000C060C060C0608031803135
:107198008031001B001B001B001B000E000E000EA0
:1071A80000040000000000000000C0C0C0C0C0C053
:1071B800C0C0C0C0C0CC804C804C805E8052805221
:1071C8008073806180610000000000000000C0C082
:1071D800806080610033003B001E000C000C001E24
:1071E800001F003B80718061C0C0000000000000EB
:1071F8000000C0C08061806100330033001E001EA3
:10720800000C000C000C000C000C000C000C000022
:10721800000000000000803F803F80010003000361
:107228000006000C000C0018001800300060807F79
:10723800807F000000000000000F000F000C000C11
:10724800000C000C000C000C000C000C000C000CD6
:10725800000C000C000C000C000F000F00000018C0
:1072680000180018000C000C000C000C00060006AA
:1072780000060006000300030003000000000000F1
:10728800001E001E00060006000600060006000696
:1072980000060006000600060006000600060006B6
:1072A800001E001E0000000C000C001E001200331F
:1072B80000338061806100000000000000000000D1
:1072C80000000000000000000000000000000000B6
:1072D80000000000000000000000000000000000A6
:1072E8000000000000000000E0FF0000000000387F
:1072F8000018000C00000000000000000000000062
:107308000000000000000000000000000000000075
:1073180000000000000000000000001F803F8061A6
:107328008001801F803F80618063807FC0380000BB
:107338000000000000000060006000600060006E57
:10734800007F807380618061806180618073007FCD
:10735800006E0000000000000000000000000000B7
:107368000000001E003F8073806100600060806143
:107378008073003F001E0000000000000000800134
:10738800800180018001801D803F80738061806161
:10739800806180618073803F801D000000000000D4
:1073A80000000000000000000000001E003F007305
:1073B8008061807F807F00608071003F001E000038
:1073C800000000000000C007C00F000C000C807F08
:1073D800807F000C000C000C000C000C000C000C52
:1073E800000C000000000000000000000000000089
:1073F800801D803F807380618061806180618073BF
:10740800803F801D80018063007F003E0000006097
:10741800006000600060006F807F80718061806123
:1074280080618061806180618061000000000000EF
:1074380000000006000600000000003E003E0006B6
:10744800000600060006000600060006000600000A
:10745800000000000006000600000000003E003E9C
:1074680000060006000600060006000600060006E4
:1074780000060046007E003C0000006000600060DE
:107488000060806100630066006C007C0076006329
:1074980000638061C0600000000000000000003E42
:1074A800003E00060006000600060006000600066C
:1074B80000060006000600060006000000000000A6
:1074C8000000000000000000000080DDC0FFC0CE0A
:1074D800C0CCC0CCC0CCC0CCC0CCC0CCC0CC0000D0
:1074E8000000000000000000000000000000006F25
:1074F800807F80718061806180618061806180614E
:107508008061000000000000000000000000000092
:107518000000001E003F807380618061806180618F
:107528008073003F001E0000000000000000000003
:1075380000000000006E007F8073806180618061C0
:1075480080618073007F006E0060006000600060F2
:107558000000000000000000801D803F80738061F3
:107568008061806180618073803F801D800180011F
:10757800800180010000000000000000000000679A
:10758800803F0039003000300030003000300030DB
:1075980000300000000000000000000000000000B3
:1075A8000000001E803F80610060007F803F8001F6
:1075B8008061007F001E0000000000000000000045
:1075C800000800180018007F007F00180018001835
:1075D800001800180018801F800F0000000000002D
:1075E80000000000000000000000806180618061F0
:1075F80080618061806180618063807F803D000060
:107608000000000000000000000000000000C06052
:10761800803180318031001B001B001B000E000EE2
:10762800000600000000000000000000000000004C
:10763800000080DD80DD80DD0055005500550077B5
:107648000077002200220000000000000000000077
:10765800000000000000806100330033001E000CB1
:10766800000C001E003300338061000000000000A1
:10767800000000000000000080618061803100335C
:107688000033001B001B001B000E000E000E001C28
:10769800007C007000000000000000000000C07FB7
:1076A800C07F800100030006000C00180030C07F76
:1076B800C07F00000000000080038007000600066D
:1076C800000600060006000E001C001C000E000646
:1076D8000006000600060006800780030006000674
:1076E8000006000600060006000600060006000662
:1076F8000006000600060006000600060006000652
:107708000038003C000C000C000C000C000C000EB3
:1077180000070007000E000C000C000C000C000C09
:10772800003C0038000000000000000000000000DD
:1077380000008038807F0047000000000000000043
:107748000000000000000000000000000000000031
:107758000000000000000000000000000010001001
:1077680000100010001000100000001000000000C1
:107778000028002800280000000000000000000089
:107788000000000000240024007C00240048007C45
:10779800004800480000000000380054005000383D
:1077A8000014005400540038001000000020005459
:1077B80000580030002800540014000800000000A1
:1077C8000010002800280010003400480048003449
:1077D8000000000000100010001000000000000071
:1077E8000000000000000000000800100020002039
:1077F80000200020002000200010000800200010B9
:107808000008000800080008000800080010002010
:1078180000100038001000280000000000000000E0
:10782800000000000000000000100010007C0010A4
:107838000010000000000000000000000000000030
:107848000000000000000010001000100000000000
:1078580000000000000000380000000000000000E8
:107868000000000000000000000000000000001000
:1078780000000000000800080010001000100010B0
:10788800002000200000000000380044004400549C
:10789800004400440044003800000000001000309C
:1078A8000050001000100010001000100000000030
:1078B8000038004400440004000800100020007C48
:1078C8000000000000380044000400180004000410
:1078D80000440038000000000008001800280028B4
:1078E8000048007C0008000800000000007C004000
:1078F8000040007800040004004400380000000044
:107908000038004400400078004400440044003837
:1079180000000000007C0004000800100010002097
:107928000020002000000000003800440044003817
:1079380000440044004400380000000000380044BF
:1079480000440044003C00040044003800000000EB
:1079580000000000001000000000000000000010FF
:1079680000000000000000000000001000000000FF
:10797800000000100010001000000000000C003093
:1079880000400030000C0000000000000000000073
:107998000000007C0000007C0000000000000000E7
:1079A80000000000006000180004001800600000DB
:1079B8000000000000380044000400080010001017
:1079C800000000100000000000380044004C005483
:1079D800005C004000400038000000000010002853
:1079E800002800280028007C004400440000000013
:1079F80000780044004400780044004400440078C3
:107A080000000000003800440040004000400040F2
:107A180000440038000000000070004800440044A2
:107A2800004400440048007000000000007C004052
:107A38000040007C004000400040007C0000000046
:107A4800007C0040004000780040004000400040BA
:107A5800000000000038004400400040005C004482
:107A68000044003800000000004400440044007C4A
:107A780000440044004400440000000000380010A6
:107A88000010001000100010001000380000000066
:107A9800000400040004000400040004004400384A
:107AA80000000000004400480050006000500048FA
:107AB8000048004400000000004000400040004032
:107AC800004000400040007C000000000044006CC2
:107AD800006C0054004400440044004400000000CE
:107AE80000440064006400540054004C004C0044FE
:107AF80000000000003800440044004400440044F2
:107B080000440038000000000078004400440044AD
:107B180000780040004000400000000000380044A9
:107B280000440044004400440054003800040000AD
:107B380000780044004400440078004800480044AD
:107B48000000000000380044004000300008000435
:107B58000044003800000000007C001000100010F5
:107B68000010001000100010000000000044004445
:107B78000044004400440044004400380000000071
:107B88000044004400440028002800280010001089
:107B98000000000000440044005400540054006CED
:107BA80000280028000000000044002800280010D9
:107BB8000010002800280044000000000044004491
:107BC800002800280010001000100010000000001D
:107BD800007C000400080010001000200040007C19
:107BE8000000000000180010001000100010001025
:107BF80000100010001000180020002000100010D5
:107C080000100010000800080000000000300010FC
:107C180000100010001000100010001000100030BC
:107C280000100028002800440000000000000000A8
:107C3800000000000000000000000000000000003C
:107C480000000000000000FE0020001000000000FE
:107C5800000000000000000000000000000000001C
:107C680000380044003C0044004C00340000000090
:107C7800004000400058006400440044006400587C
:107C880000000000000000000038004400400040F0
:107C98000044003800000000000400040034004CD8
:107CA80000440044004C00340000000000000000C4
:107CB80000380044007C0040004400380000000008
:107CC800000C0010007C00100010001000100010C4
:107CD80000000000000000000034004C0044004494
:107CE800004C003400040078004000400058006454
:107CF800004400440044004400000000001000005C
:107D080000700010001000100010001000000000AB
:107D1800001000000070001000100010001000108B
:107D2800001000E000400040004800500060005093
:107D3800004800440000000000700010001000100F
:107D480000100010001000100000000000000000EB
:107D580000780054005400540054005400000000FF
:107D6800000000000058006400440044004400443F
:107D780000000000000000000038004400440044F7
:107D880000440038000000000000000000580064B3
:107D98000044004400640058004000400000000017
:107DA8000034004C00440044004C0034000400043B
:107DB80000000000005800640040004000400040FF
:107DC80000000000000000000038004400300008F7
:107DD8000044003800000000002000200078002047
:107DE8000020002000200018000000000000000013
:107DF8000044004400440044004C003400000000EB
:107E0800000000000044004400280028002800105A
:107E18000000000000000000005400540054006CF2
:107E2800002800280000000000000000004400288E
:107E380000100010002800440000000000000000AE
:107E480000440044002800280010001000100060C2
:107E580000000000007C0008001000200040007CAA
:107E68000000000000180010001000100020002082
:107E78000010001000100018001000100010001072
:107E8800001000100010001000100010003000104A
:107E9800001000100008000800100010001000304A
:107EA8000000000000000074004C0000000000000A
:107EB80000000000287F0008F52B000800000000E3
:107EC800000000008000000000000000000000002A
:107ED800807F00080A28000000000C4200008C4245
:107EE800887F00080E3C00000000F041000082423C
:107EF800907F000808190000000020420000A042FE
:107F08000000000000000000010203040607080941
:107F1800000000000102030449444C450000000031
:107F280064656661756C745461736B0050313A25F1
:107F3800336400000000000050323A25336400002A
:107F4800573A257320413A2533640000445241577B
:107F58000000000050322057494E5300503120573E
:107F6800494E5300303D72657374617274000000AD
:107F780047616D65000000004E4F524D0000000043
:107F880042494720000000004D494E4900000000CA
:107F98004572726F7220777269746520706F6C61B8
:107FA800726974790A0000004572726F72207772E4
:107FB800697465206F75747075740A004572726F04
:107FC8007220777269746520696E69740A0000000E
:107FD8004572726F7220777269746520636F6E667E
:107FE80069670A0052656164206572726F720A00DF
:107FF800232D302B2000686C4C006566674546478A
:10800800003031323334353637383941424344450C
:10801800460030313233343536373839616263647B
:1080280065660000000FC93F000F494000CB96402D
:10803800000FC9400053FB4000CB164100ED2F4113
:10804800000F49410031624100537B41003A8A41A7
:1080580000CB9641005CA34100EDAF41007EBC41DE
:10806800000FC94100A0D5410031E24100C2EE41F4
:108078000053FB4100F20342003A0A4200831042D7
:1080880000CB164200141D42005C234200A5294281
:1080980000ED2F4200363642007E3C4200C7424285
:1080A800000F4942A2000000F90000008300000010
:1080B8006E0000004E0000004400000015000000A3
:1080C80029000000FC000000270000005700000005
:1080D800D1000000F500000034000000DD000000C1
:1080E800C0000000DB0000006200000095000000F6
:1080F800990000003C0000004300000090000000D0
:1081080041000000FE000000510000006300000074
:10811800AB000000DE000000BB000000C50000004E
:1081280061000000B7000000240000006E0000009D
:108138003A000000420000004D000000D20000009C
:10814800E000000006000000490000002E000000CA
:10815800EA00000009000000D100000092000000C1
:108168001C000000FE0000001D000000EB000000E5
:108178001C000000B100000029000000A70000005A
:108188003E000000E800000082000000350000000A
:10819800F50000002E000000BB00000044000000B5
:1081A80084000000E90000009C000000700000004E
:1081B80026000000B40000005F0000007E00000000
:1081C800410000003900000091000000D6000000C6
:1081D800390000008300000053000000390000004F
:1081E800F40000009C000000840000005F00000014
:1081F8008B000000BD000000F9000000280000000E
:108208003B0000001F000000F8000000970000007D
:10821800FF000000DE0000000500000098000000DC
:108228000F000000EF0000002F0000001100000008
:108238008B0000005A0000000A0000006D000000DA
:108248001F0000006D000000360000007E000000E6
:10825800CF00000027000000CB000000090000004C
:10826800B70000004F000000460000003F0000007B
:10827800660000009E0000005F000000EA000000A9
:108288002D0000007500000027000000BA00000063
:10829800C7000000EB000000E5000000F10000004E
:1082A8007B0000003D0000000700000039000000CE
:1082B800F70000008A000000520000009200000051
:1082C800EA0000006B000000FB0000005F000000F7
:1082D800B10000001F0000008D0000005D000000DC
:1082E80008000000560000000300000030000000F5
:1082F80046000000FC0000007B0000006B0000004E
:10830800AB000000F0000000CF000000BC0000003F
:10831800200000009A000000F40000003600000071
:108328001D000000A9000000E3000000910000000B
:10833800610000005E000000E60000001B00000075
:10834800080000006500000099000000850000009A
:108358005F00000014000000A0000000680000009A
:10836800400000008D000000FF000000D800000061
:10837800800000004D00000073000000270000008E
:108388003100000006000000060000001500000093
:1083980056000000CA00000073000000A80000009A
:1083A800C900000060000000E20000007B0000003F
:1083B800C00000008C0000006B0000000000C93FF6
:1083C8000000F0390000DA370000A2330000842EE4
:1083D8000000502B0000C2270000D0220000C41F5C
:1083E8000000C61B0000441704000000070000003E
:0483F8000900000078
:0883FC00D47DFF7F01000000A9
:04840400B5010008B6
:0484080091010008D6
:10840C000100000010000000AAAAAAAA101A00007D
:10841C00A85600080B120000F4690008070A0000B7
:10842C00507700080000803F0024F400300000204A
:10843C0000000000C845002030460020984600206F
:10844C000000000000000000000000000000000020
:10845C000000000000000000000000000000000010
:10846C000000000000000000000000000000000000
:0C847C00000000000000000000000000F4
:04000005080041D1DD
:00000001FF
